:020000041100E9
:10300000002373B52B4D2C4C28006361022601F080
:103010006FF94021FE2221742800284B009601F010
:10302000B9F9002836D1217CFF222800244B0096D4
:1030300001F0B0F900282DD1224BA2899A4226D165
:10304000E389214A93420DD1204B6361204B2268D2
:10305000002A03D1002B01D043CB43C4280001F048
:1030600085F973BD1B4A934201D00023EFE71A4B49
:103070001A4A1B68934206D9C02304222800217CE7
:103080009B0001F0FDF9114B6361154BDFE7002355
:103090002374EAE7CC233821AC2228009B01217459
:1030A00001F0EEF90028F2D10E4B63610E4BE38183
:1030B0000E4BCCE7F441FF1F9C61FF1FA861FF1F6F
:1030C000AA61FF1F59590000830500001D4100112E
:1030D00024BD001182150000C061FF1F871300008E
:1030E00030BD0011D5410011AAAAFFFF18BD001183
:1030F000F7B5164B0192C318021D002000938823D8
:103100005B05D3181B685C1C1AD09CB2402C18D8E5
:103110008D781E0CAC466746CD782D023D43AE42FD
:1031200006D1019800280ED110000C70240A4C70B2
:1031300003249BB20733A343D218009B9A42DED3E9
:10314000FEBD4432F9E71000FAE7C046FC0F00006C
:10315000802213B503000324019189B25201073183
:103160009B18A14304305A1A88235B05C3181B68B7
:10317000591C03D190429241104016BD99B240298A
:1031800007D80B000733A343C0189042ECD30020AC
:10319000F3E74430F9E7134B134A1B68126810B584
:1031A000FA24934201D81A00F824104BE4021B6859
:1031B0009A4210D813000E4A12689A420ED3013375
:1031C00007D1F823DB029C4203D10A49054808F0E5
:1031D00037FB200010BDFC24E402ECE7FE24E402EF
:1031E000F7E7C04600C0071100D0071100E0071143
:1031F00000F00711FFFFFF7FF0B59BB015000490B2
:103200000391402A00D9A0E006AB59801A80FFF74D
:10321000C2FF0400042816D9002206A9FFF768FFA0
:10322000052810D906AB1B88AB420CD1002D07D066
:10323000514B2A000499C01808F052FC002802D112
:1032400001201BB0F0BD06AB1D8020000699FFF7E2
:103250007FFF041E7BD1069B0793FFF79CFF802313
:103260005B01C618802307001B039E4201D3F8268A
:10327000F60288235B05F31801931B68013302D023
:10328000019808F07DFC3D49019808F0D9FA3B1DF2
:103290000293331D05938822029B52059B181B68DD
:1032A00008935A1C3CD044219AB20091402A04D879
:1032B0000320D11D814389B2009103991B0C8B42DD
:1032C00024D0402A22D80122300008A9FFF710FF9D
:1032D000021E1BD1380008A9FFF70AFF04000428CA
:1032E00031D9009A059B9B1880225201B218934253
:1032F00040D288235B05C118009A09A808F0B8F9E4
:103300001D4B009A09A9F01808F06AFB009A029B6D
:103310009446634402931A4B029AFB189A42BAD31A
:1033200088235B05FC1821680198013908F088FAA8
:10333000200008F025FC039A07AB5A80300007995B
:10334000FFF706FF0400002C03D1002079E70428D2
:10335000FBD988235B05E018069908F071FA03236E
:10336000EA1C9A4300D16BE7034B0499E01808F07C
:1033700037FB65E70424ECE704000011FFFFFF7F43
:10338000F80F0000F7B505001400402A21D80027E7
:1033900001AE71803780FFF7FEFE042816D93A008F
:1033A0003100FFF7A5FE042810D93688BC420BD0A7
:1033B000BD4209D0221CB44200D9321C064B92B245
:1033C000C118280008F054F930B2FEBDC04300B265
:1033D000FBE703204042F8E70400001137B5042260
:1033E00004000D0001A81649FFF7CCFF02000428D5
:1033F0000BD1019BA34208D3AB4204D0104901A8D2
:103400000195FFF7F9FE01203EBD0E4C2368200018
:10341000019308F0B5FB019920000139019108F0F2
:103420000FFA80235B01E418074B9C42EED1042283
:10343000034901A80195FFF7DFFE0020E4E7C0463D
:103440005555000000C007110000081130B589B0C3
:1034500008F03EFA10226946254808F0D1FB254BBA
:10346000009A9A420ED1019B029A0F2B33D8002169
:1034700001240698013B08D2002900D00292029B49
:10348000013331D10023029325E0551CF2D1020013
:103490002100EFE710341022200004A908F0B0FB4F
:1034A000029B013301D1069B0293882304995B059B
:1034B000C918059B06981A03120B049105928142C4
:1034C00003D02B4201D108F0D3F8019B013B0193BB
:1034D000019B002BDED1029B002B03D004930498A8
:1034E0004168084709B030BDE025014C2D03EFE7E6
:1034F00000000111504859368022F8B5964C974B80
:10350000D200002120001C6008F0B2F92300944A88
:1035100088331A60934B1A786A23002A00D011333B
:10352000E3620A232365904B37221B780820A363AC
:103530008E4B2118E361102323628D4B3B25636181
:10354000C823DB00A36123008C331A602823013ACF
:10355000E26320646364CA67043A211DCA672100DC
:10356000BC310D602100C03108602100C4310B6006
:1035700021000635CC310D602100083DC8310D60B9
:103580002100D0310A602200D43210602200D832EB
:10359000136022000227E032210017604222DC3152
:1035A0000A6021001B3DE4310D602100E831086014
:1035B0002100EC310B6023000521F4331960230056
:1035C000F0331A602300183290331A6023009433CA
:1035D000186023001E3A98331A60AF23DB00236083
:1035E000644BFA262363644B644DE360644BF03113
:1035F000A3642300FF31FC33B600A16021611E608B
:10360000A5627325E5656D3D6565A56596255D4AF1
:10361000AD00E264666258606766A566002709250A
:10362000A767E566584F594D606720002567E26738
:103630003A6015279C30676007001A203860200028
:10364000A0300700212038602000A83007004C4837
:1036500038602000F830066026006427A436376002
:1036600026005F3FAC3637602600033FB036376038
:103670002600C637B436376026000027B8363760D4
:1036800038269E60424E96205E64424E5A66DE6147
:10369000414E9A645E62F53EFF3E9E621E269A6728
:1036A000354A8000DE661F675F67DD651D6618624C
:1036B000DA67BE23394A5B00E250394BD8382350D1
:1036C00004302250C4225200A350C623E4205B00E1
:1036D000E1500433334AE1503349344BD16034492B
:1036E000800019503349E938FF3819503249043005
:1036F000195032493248D16132491163324951631C
:103700001900F4310860CE20304940001160304982
:10371000195019002F48F83108602F49D1658221CE
:103720002E4A89005A501A002D490832D1671A00D2
:103730002C49B432116088212B4A89005A501A0052
:103740002A49883211602A4ADA6407F0D9FF012039
:1037500008F0B6F8F8BDC0460004FF1F4064FF1F24
:10376000206FFF1F3044FF1F4A0AFF1F3A07000067
:1037700080C3C9019A020000DC0500006A1800003D
:1037800050C3000088130000F009FF1F204E000006
:103790006509FF1F68100000C409000040420F00C7
:1037A00010270000FC00FF1FC11BFF1F0000FF1FB0
:1037B000152CFF1FA52FFF1F3D2EFF1F811FFF1F71
:1037C0007126FF1F9D1FFF1F4921FF1F0D1FFF1F98
:1037D0009528FF1F7D29FF1FD918FF1FA127FF1F55
:1037E000C524FF1FD124FF1F0D1EFF1FC51EFF1F75
:1037F000851DFF1F0223F0B50124614D614E2B7022
:10380000614B91B01C70614F039333680021082015
:10381000FB7006F0DFFD082006F0D6FC002398427E
:1038200005D0FA78552A02D0332A00D09BE03360C5
:10383000042006F049FF08F0C3F8FFF75DFE07F02B
:103840002FFF1F2201240021514B10AE1A70514B43
:103850001C70514B1970514B19689143163A0A4329
:103860001A60602219689143403A0A431A6008F0CE
:1038700067F908F055F8C120FF21494B80001A581C
:103880008A431A50C522920098588843BF39014391
:1038900099509858434908408021C901014380202C
:1038A00099509958C0050902090A0143995080218D
:1038B0003D48490107F05CFF032322003B49019486
:1038C00000933B4807F0F4FF2C223A4905A807F083
:1038D000CFFE05AC61782078023406F095FCA64254
:1038E000F8D1354C0020012106F0A2FD2268334BAF
:1038F00003201A40A023DB021343236080232268A5
:103900009B041343236022682D4B1A4080239B03A2
:10391000134323602B4A2C4B934200D8012008F01C
:103920000FF808F015F880232268DB0413432360A6
:10393000287807F085FE039B1878C0B208F018F8C5
:1039400007F036FF2149042008F0B2F806F088FE9F
:1039500000F0A8F800F0EAFD00F092FE00F00CFA8A
:10396000002011B0F0BD00932100184A042007F098
:10397000F7FF8023DB059C62FFF768FD58E7C04630
:103980004A0AFF1F34F000403044FF1FCC61FF1F84
:10399000480AFF1F490AFF1F680AFF1FBCF00040CA
:1039A00000E100E0FF00FFFF3444FF1FB856FF1F97
:1039B0003454FF1F40BC001114F00040FF7FF8FF9B
:1039C000FFFF9FFF0080FF1F206FFF1F3B000108CC
:1039D00070B500252549264A26484D6308CA1B05AF
:1039E0001B0DED188242F9D100268022224B920550
:1039F0008B630921214B224C1E62224B1120DA6776
:103A0000214BDA688A43DA609A6820490A409A6052
:103A1000266008F07DF8112008F0BAF88022636C67
:103A200093436364EE24E4006C43194A200C0400C1
:103A3000642390420AD8FA223300D200904205D97A
:103A4000144B0A21C01807F0CBFDC3B2124A112053
:103A50001372D48007F0E4FD104B1B78002B04D1C7
:103A60000F4B1021187808F083F870BD0000054056
:103A70008805054000060540FF01000000F00040F9
:103A80000038004004E100E03CF00040FFDFFFFFB1
:103A9000B70B000030F8FFFFB461FF1FEE63FF1F9C
:103AA000EC61FF1F002210B51100112007F0A0FFEC
:103AB00010BD0000F8B500230926374F374C3B6294
:103AC000E3681120B343E36008F062F8112008F0C6
:103AD0001FF8112008F064F8402322688025134362
:103AE000236080236268DB0213436360A3682C4A6F
:103AF0002B43A360A36802211340A3608023A26824
:103B00009B0113431022A360236C0720934323647B
:103B1000236C0F3A1343236480235B003B62226BC8
:103B2000204B1A402263626B1A406263A26B1A40F8
:103B3000A263E26B1340E363E3681B4A1340E36054
:103B400006F062FB0121072006F072FC174B1120E2
:103B50005A6C15435D6407F0BBFFFD21144B154AF9
:103B600089005A508023C720626B5B031343636351
:103B7000E36880003343E3600F4B104A195811404B
:103B8000802212020A431A50802292051A600822EB
:103B90000B4B5A63F8BDC04600F000403CF00040BB
:103BA000FFFFDFFFEFFFEFFFFFFF7FFF0038004069
:103BB0000000FF1FD139001100E100E0FF00FFFF0E
:103BC0000000054030B503A804880B20002C0ED15E
:103BD0004968074D08784978090201430A20A9423B
:103BE00005D1012120001980024B1B7A137030BDD2
:103BF000192A0000B461FF1FF7B5150008AA16883E
:103C00004A680F4F14785278120222430A24BA42AB
:103C100014D10122DBB2019200962A0007F070FC59
:103C2000041E0BD1074B1B68002B07D068782A783D
:103C30000002104342425041013098472000FEBD2F
:103C4000022900003861FF1F30B501250379040007
:103C5000BFB02B4211D00A49408806F0BDFF284270
:103C60000BD0084B01A95B8D4D800B80064B0022C9
:103C70001B7A60880B7104F08FF83FB030BDC046EE
:103C80003061FF1F6840FF1FB461FF1F10B5054979
:103C9000054806F057FF0421044A054806F014FFC2
:103CA00010BDC0463061FF1FFFFF00006CBC00115B
:103CB0006840FF1F10B5024804F0F0FE10BDC0467A
:103CC000493C0011062310B5837010330371443B47
:103CD00043712A3383714433C371002302220121CB
:103CE00003720E4B027041701C8881724472197A03
:103CF0000273C1729A784273DA7882730322C273B4
:103D00001A7902745A7942740C2282749A79C274B4
:103D1000DB7903751123C370152010BDB461FF1F3B
:103D200010B5142007F074FD124B14220021186006
:103D300007F09EFD002007F04BFE012007F078FF02
:103D4000022007F06DFE032004F04CF9042006F079
:103D500061F9052003F08AFB062004F057F80720DC
:103D600001F05AFA082006F08FFE092001F034F81D
:103D700010BDC0463C61FF1F07F0F2FE012007F0B6
:103D800027FD07F0DDFC0000094B10B50400984248
:103D900005D0012904D12000064906F0D3FE10BD4C
:103DA0000229FCD1013904F037FE0028F3D0F6E7F0
:103DB000FEFF00006261FF1F70B50D7A100004AABB
:103DC0002C00168810221440154220D1002E20D13C
:103DD0000A78022A18D14A68517815780E4A0902E1
:103DE0002943914205D00D4A914209D01C800A24F2
:103DF00004E014220A491A8007F03AFC200070BD42
:103E00000C2208491A80F7E71C800124F6E70824F1
:103E1000F4E70B24F2E7C046F3FF0000F4FF0000D4
:103E2000BC42FF1F48BD001110B5040007490848F7
:103E300006F088FE074804F071FD0020E40704D571
:103E40000721054A054806F03FFE10BD6261FF1FCD
:103E5000FFFF0000893D0011B0BC0011AC40FF1F06
:103E600000B50C4BBFB01A780B4902A800F0C2FC99
:103E70006B4680B2D880002809D06A46074B01A95A
:103E80001B889380064B0022188803F085FF3FB003
:103E900000BDC0464061FF1F4161FF1F0641FF1F7B
:103EA0001042FF1F00B50C4BBFB01A780B4902A897
:103EB00001F0B8FE6B4680B2D880002809D06A466F
:103EC000074B01A95B8D9380064B0022188803F0F5
:103ED00063FF3FB000BDC0466A61FF1F6B61FF1FFB
:103EE000AC40FF1F1042FF1FF7B50E00377A1C00D1
:103EF00008AB11003D001A8820231D401F423CD111
:103F00003378022B3BD173681F785B781B023B43ED
:103F10001E4FBB4208D01E4FBB4214D01D4DAB42BA
:103F200021D00A252800FEBD002A2AD1142C2AD827
:103F30002200F06807F09CFB174B1C70012CF1D994
:103F4000FFF7B0FFEEE7002A1BD1202C1BD8220080
:103F5000F06807F08DFB114B04211C70104B187892
:103F600007F006FEDEE7E3B20124009201940A00A6
:103F7000310007F0C5FA0500D4E70825D2E701258E
:103F8000D0E70B25CEE70D25CCE7C046F3FF0000B8
:103F9000F4FF0000022900006A61FF1F4061FF1F5B
:103FA000EC61FF1F332310B5040003700A22074998
:103FB000013007F05DFB064B0F201B681A0AE37205
:103FC00022731A0C1B0E6273A37310BDB461FF1F22
:103FD000DC61FF1F30B5012503790400BFB02B421F
:103FE00013D00B49408806F0F7FD28420DD06A46F1
:103FF000084B02A81B889380FFF7D4FF6B46D8803C
:104000000022608801A903F0C7FE3FB030BDC04662
:104010006261FF1F0641FF1F10B5024804F03EFD1C
:1040200010BDC046D53F001170B5160004AA148813
:1040300005AA15784A685078117800022A4A084380
:10404000801805284BD807F023FB03131E29343FA3
:104050000720032C0BD80422121BAA4200D92A00E5
:1040600022491A803000091907F002FB002070BDB8
:104070000720112CFBD81222121BAA4200D92A00B9
:104080001B491A80EEE707200E2CF0D80F22121BD6
:10409000AA4200D92A0017491A80E3E70720032C17
:1040A000E5D80422121BAA4200D92A0012491A801C
:1040B000D8E70720032CDAD80422121BAA4200D921
:1040C0002A000E491A80CDE70720032CCFD80422FE
:1040D000121BAA4200D92A0009491A80C2E700220D
:1040E0000A201A80C3E7C046DCD5FFFFFBBC0011E5
:1040F0008861FF1FEBBC0011E6BC0011E1BC0011A0
:10410000DCBC001110B50D21024A034806F0DCFCAE
:1041100010BDC046D0BC00111C41FF1FF0B50024EB
:10412000274E85B03000B47100F0E2F8254D264BE3
:10413000EA89297C9A422FD10423300003AA00F097
:1041400057F90400300000F011F90123B371002C7D
:1041500034D16B4699892B68C9BA4B4329891B4ACC
:104160001B145B1853806B46D9896B6849BA89B2B6
:104170004B4369891B0C5B181548191C1BB2834201
:1041800000DD011C0B0400D5002113889180013350
:104190001380200005B0F0BD0227220003AB3000E1
:1041A000009700F0F7F80E230400297C012230006C
:1041B00000976B4400F0EEF80443C3E71C00E8E707
:1041C000F441FF1F9C61FF1F83050000B461FF1FC6
:1041D0000F27000073B5234E300000F089F8224D00
:1041E00007236A463000297C00F002F90400300001
:1041F000002C33D16B461B787F2B2FD800F0B6F8FC
:104200006B46D878F02302041B031A406B469B8848
:1042100016495BBA9BB21A432B68000953432A899B
:104220001B0C9B184B806B465A789B7812031B0122
:104230001A436B68024353436A891B0C9B180C4852
:104240001A1C1BB2834200DD021C130400D500229D
:104250000B888A8001330B80200076BD00F086F841
:104260000124F9E7F441FF1F9C61FF1FB461FF1FA8
:104270000F27000070B5114C237C002B0FD0382B7A
:104280000ED10F4D280000F033F8CC23AC222800CB
:10429000217C9B0100F0F4F8280000F067F870BD65
:1042A000084BE2899A42FAD1054D280000F020F827
:1042B00000222800217C00F0C5F8EDE79C61FF1F7B
:1042C000F441FF1F8305000010B5084B1A7C002A3B
:1042D00009D05B69002B06D09847041E01D0FEF779
:1042E0008FFE200010BD0124F9E7C0469C61FF1F2E
:1042F00070B5C17905000C00631E9C411A4BE402A5
:10430000E41849000460C9B2007906F0C7F8E979F9
:10431000687949000131C9B206F0C0F8E87909307E
:10432000C0B207F03DFC0023E36661332360AA7945
:104330005B3B002A0ED022689A43023B1343236062
:104340000A23E3610733236200232363A36301335A
:10435000E36370BD22689A4302231343236046231C
:1043600063610633A361EFE70050004070B500259C
:1043700004000368DD66C0790930C0B207F008FCAC
:104380002900207906F026F82900607906F022F845
:1043900070BD0000F8B51E0006AB1D780023046850
:1043A0001700E366616007F093FA01238022E36659
:1043B0002B0027615200013B08D207F081F9082049
:1043C0000A4A1168002D03D12800F8BD2261F2E7E6
:1043D000236F034203D02369013D33700136136814
:1043E0005B1A032BEED90125EEE7C0466008FF1FDC
:1043F00070B51C00002305681600EB66696007F0C5
:1044000067FA01238022EB6623005200013B08D2A9
:1044100007F056F908200A4A1168002C03D1200041
:1044200070BD2A61F2E72B6F034203D02B69013C78
:104430003370013613685B1A032BEED90124EEE7C3
:104440006008FF1F002370B504681500E366616013
:1044500007F03EFA0123E366256107F031F9802079
:10446000064A80001168636B034205D113685B1A2A
:10447000032BF8D9012070BD0020FCE76008FF1F66
:1044800070B51D00002304681600E366616007F044
:104490001FFA0123E36626610F33626B1A42FCD0D8
:1044A0002B0A23611023626B1A42FCD0EDB2256106
:1044B00007F006F98020074A80001168636B034209
:1044C00005D113685B1A032BF8D9012070BD0020B9
:1044D000FCE7C0466008FF1F70B51E00002305689A
:1044E0001400EB66696007F0F3F90123A619EB6687
:1044F0000F33B4420ED107F0E3F880200A4A80005F
:1045000011686B6B03420CD113685B1A032BF8D94B
:10451000012070BD21782961696B1942FCD00134FA
:10452000E7E70020F5E7C0466008FF1F10B5084C1C
:10453000E368002B08D18022064B52021B689B18AF
:104540006360054B1B68236007F022FAA06010BD72
:10455000DC61FF1FC8F00040CCF0004070B5184A85
:10456000936A916A9942FBD116498A689A421FD38D
:104570009A1A8B60144B0126186893B2D202D20E9D
:104580004343424300204C681B0A1B1912029B182C
:104590000E4C0A684B60551CA3420CD8002801D071
:1045A0004B600A600A4A136008680A4B186070BDC5
:1045B000581E821ADDE7084A30009B182A00EAE7F5
:1045C00000F00040DC61FF1F140AFF1F40420F0093
:1045D000C8F00040CCF00040C0BDF0FF70B51F4CEB
:1045E00023793F2B01D93F2323711D4B22791A7068
:1045F0001878C0B207F08CF818231A491A4A0B80B1
:104600001A4913800B805380A379194980200B80AD
:104610000C21938001334B43164D191C000183423A
:1046200000D9011C2980D1806379002B11D101337D
:104630006371237A012B01D8022323726279237AD2
:104640000D4853430A21584306F0CAFF0B4D28601A
:1046500070BDA02BEDD9A023EAE7C046D061FF1FB3
:10466000480AFF1F0E42FF1FDC43FF1F0C42FF1FC3
:104670000A42FF1F0842FF1F71020000C061FF1FB6
:10468000F8B514210020FEF7A9FE114C011E114DB2
:1046900009D10C22104BC1CBC1C4280007F0E8F8A7
:1046A000FFF79CFFF8BD0C2220000C49FEF76AFEC4
:1046B0000C2802D0084B43CB43C40C2228000849E5
:1046C000FEF760FE0C28EBD00C220021E5E7C04687
:1046D000D061FF1F9C61FF1F3CBD0011FC0C00005E
:1046E000F50C0000F0B51D4C8022A5440400882084
:1046F00069465201400507F013FA902212016A44FC
:104700001300200032C832C316C816C38023144CCD
:10471000144FA6689B033343A3603B6007F0A0F8E7
:104720008823A0685B05C01807F02AFA00258823B3
:1047300029008022A0685B05C01840196944520016
:1047400007F04EF980230135FF355B019D42EED124
:10475000A6603E60044B9D44F0BDC046FCEFFFFFE9
:104760004C43FF1F9808FF1F04100000F0B5040021
:1047700087B0002825D0684607F06AF91B4C02284C
:1047800006D106226946200007F0AAF9002816D0B3
:104790006946002301250F262F00E25C0133100932
:1047A0001030874038002F00324097403A000243D3
:1047B0004A610439062BEFD16846FFF793FF07B033
:1047C000F0BD182269460A4807F0AAF96A46A30014
:1047D000D358013305D01822FF21684607F048F866
:1047E000EAE70134062CF1D1E9E7C0466509FF1F6D
:1047F00000090011F0B5002504000E0085B0AA42A2
:1048000000D186E04B1C087801934B788978377982
:1048100009021943F3783F061B040B431F43039718
:1048200020706570252800D196E033D8112813D860
:1048300007F02EF869002501250125012501AA00B0
:10484000B800B1002501250125012501250125011B
:104850002501250105011F01232800D1DEE0DB2809
:1048600000D02EE1042A00D8ACE01025052A05D09E
:10487000551F2A003800711D06F0FAFE052231008E
:10488000200006F0F5FE2A003900601D06F0F0FE5B
:1048900005353EE0562859D010D8332800D19DE088
:1048A000552839D02628DAD19C4B2900132218002C
:1048B0001D0006F0DDFFFEF7A3FB5CE0712800D1D0
:1048C00077E0722800D180E0602800D18BE0DC28FE
:1048D000C5D1022A00D875E07378BFB26370B3788F
:1048E000A370032A05D0033A390092B2F01CFEF7F8
:1048F00083FC10223900E01CFEF744FDC51C002893
:1049000007DA60705CE00C222000854906F0B0FEFA
:104910000C25280005B0F0BD013A824D0C2A13D8B1
:10492000002A0AD02800019906F0A2FEFFF756FEE1
:104930000C2228007C49FEF75FFC29000C22601C39
:1049400006F096FE0D25E4E70C22EBE7754D774B5C
:104950002A0043CB43C2E9E7013A704D0C2A11D833
:10496000002A08D00199280006F082FE0C222800B7
:104970006F49FEF741FC29001322601C06F078FE07
:104980001425C6E70C22EDE705226A49601C06F0F3
:104990006FFE0625BDE712226749601C06F068FE1F
:1049A0001325B6E708226549601C06F061FE09255B
:1049B000AFE77178F02905D8614B188801F08EFDBA
:1049C0000225A6E7FF236370FAE75E4B012A03D0B6
:1049D00072789A706270F3E79B78F4E72000FFF733
:1049E000E1FA050095E7013A564B574D062A10D8D3
:1049F000002A10D0012128005970019906F038FED4
:104A000001F042F829000622601C06F031FE07255D
:104A10007FE70622EEE700225A70F3E7042A04D962
:104A20004A4D2F6006F0B4FFA860FFF797FD0422FF
:104A3000039003A9601C06F01BFE052569E7444DA1
:104A4000062ADFD906222800019907F049F8002834
:104A5000D8D006220199280006F00AFE06223D4918
:104A60002800FEF7C9FB0123364A91780B43937067
:104A7000C8E7012AA6D07078FFF778FEA0E70128E2
:104A800000D0ECE6931E344F1A2B04D87378002B19
:104A900009D100F015F9314B39001D78601C6A1EF0
:104AA00006F0E6FD35E7551E2A000199380006F0AC
:104AB000DFFD2B49AAB23800FEF79EFB00F036F965
:104AC000E9E7DA281DD1042A00D87BE7082A15D99E
:104AD000B37972791B021343F27912041A43337AC1
:104AE0001B0613433B603B68052231002000039303
:104AF00006F0BEFD0422601D03A956E7FE23637085
:104B0000F1E7DE2800D05DE7511E012A01D1002522
:104B1000FFE6019800F09EFFF9E7C0469C61FF1F89
:104B200048BD0011D061FF1FFC0C00003CBD00110E
:104B3000F50C0000A861FF1F8861FF1F5043FF1F95
:104B40001042FF1FCC61FF1FAD42FF1FDC61FF1F42
:104B50006509FF1FADAC0000CD63FF1FCB63FF1FD6
:104B6000AEDE000070477047020010B5094B0A32F4
:104B7000094C92B2DA815A8298811882207802F028
:104B800013FB0422054B012120781A7006F0F0FF78
:104B900010BDC046DA42FF1F1664FF1F1564FF1FD9
:104BA000013870B5042809D806F072FD03092808F9
:104BB0001200234B0221187806F0DAFF70BD204B5B
:104BC0000821187806F0FCFF00221E4B1A72F5E748
:104BD000802200241B4B1A4D52001A8108211A68AA
:104BE0002878DC7206F08CFF2100287806F0E0FFC0
:104BF000012000F067FE00F047FFDFE7104B0821BF
:104C0000187806F0DDFF1048FFF75CF80F4B104AEC
:104C10009B79002093800F4A13808022094B520019
:104C2000D8721A8100F04EFE00F02EFF0A4B9B78DE
:104C3000002BC3D0094A136006F022FFBEE7C0462E
:104C4000EC61FF1FC061FF1F1942FF1FD061FF1FF2
:104C5000DC43FF1F0A42FF1FCC61FF1F34F00040FE
:104C600010B501290BD1082809D1054B1B78002B61
:104C700005D02622034B04485A72FFF775FF10BD7A
:104C8000EE63FF1FC061FF1FC40900000300F0B501
:104C90000A4D8E18B14202D152008018F0BD0C7836
:104CA0002F6824093C5D0F271C700C7801313C40B3
:104CB0002F683C5D5C700233ECE7C0460442FF1F86
:104CC0000D22114B10B51A700C23104C1049237093
:104CD000093A033B0F48637006F0CAFC2D230122FA
:104CE0000D490E48A371FFF7D1FF01220C49FFF7D0
:104CF000CDFF01220B49FFF7C9FF00220A4910002E
:104D0000FEF77AFA10BDC046EA63FF1FCB63FF1FB0
:104D1000FBBC0011CD63FF1F6709FF1FD263FF1F9C
:104D20006609FF1F6509FF1FAEDE000070B5124C5B
:104D3000132220001149FEF725FB114D002817DD35
:104D4000AB78002B14D0431C2B7009236B7000230D
:104D500000190370287829000130C0B206F010FD58
:104D6000297822000139C9B2002005F0CBFD70BDC1
:104D7000FFF7A6FFEEE7C046CD63FF1FAEDE0000E3
:104D8000CB63FF1F10B5114B1A781870002A0ED094
:104D900000280BD10E4B1A78062A07D85423D3408B
:104DA000DB0703D50B4B187802F0FEF910BD002885
:104DB000FCD0074B1B78012B02D0033B022BF5D80C
:104DC000044B0121187806F0D3FEEFE7EE63FF1FD6
:104DD0001564FF1F1664FF1F70B5514E514A5249AA
:104DE0003070082005F01AFC0121022005F020FB9C
:104DF000022005F001FC0121002005F019FB002034
:104E000005F0FAFB00F0AAFEFEF7FAF806F0E8FE5D
:104E1000032246494648FFF739FF2D2403000422A8
:104E20001C7044490130FFF731FF30230470424DBC
:104E3000424C437083702E3B062220004049EB8792
:104E4000FEF7A0FA062813D0200006F001FE022883
:104E500009D00321200006F0EBFB8D23E3706E3BAD
:104E6000237119336371062220003549FEF7C4F916
:104E7000344B1B68FC335C64FFF758FF0020FFF7DE
:104E800081FF314C314A0121314B1278207802F0F8
:104E90004DF9304A304B12780021207802F046F963
:104EA00001222E4B1A702E4BDB78552B31D12D4B16
:104EB0003B325A722C4B2D4AAB81EA812B826A829B
:104EC0002021307806F04CFC0120404205F066FDC0
:104ED0000120404205F002FEFFF714F9FEF7D6FE6E
:104EE00000F0A4FC01204042FEF79EFF012006F0E6
:104EF000EFFBF02001F0D6FA0121307806F038FE01
:104F0000307802F0ADFA1A4806F002FDFEF7D2FD45
:104F100070BD6422174B5B7953431A000A32CBE70A
:104F2000EC61FF1F654B0011614C00115043FF1FE6
:104F30008861FF1FA861FF1FDA42FF1F6509FF1F7D
:104F4000ADAC00004064FF1F1664FF1F3842FF1F16
:104F50001942FF1FEA63FF1FCB63FF1FBC63FF1FE4
:104F6000CC61FF1FC061FF1FC4090000CE09000013
:104F7000EE61FF1FD061FF1FF8B50A0020230D006E
:104F80001A40194257D0574B1B78002B50D0FFF7CF
:104F9000E5FA554B554C564E99686268737A8A1AF1
:104FA000DB039A4202D36160FEF784FD327A217AF4
:104FB000531EDBB2994205D1FFF75CF9002000F0E7
:104FC00099FD0FE09142F9D300232372FFF77CF99A
:104FD000012000F08FFD474F3800FEF773FE3900C7
:104FE00006F01EFE637A002B1FD0013BDBB263721A
:104FF000002B1AD1404BDB78552B01D106F040FD38
:10500000E37A002B0CD000233C4A3A4FE37213881A
:10501000380001331380FEF755FE390006F000FE1C
:10502000642370795843FFF79FFD237A013323727D
:1050300020206840F8BD0BB2002B0ADA304B1878FC
:1050400006F03EFD002801D006F0C2FD80200002DF
:10505000EFE70224214206D0244B01201A72FFF709
:1050600091FE2000E5E70B071ED5FFF777FA1E4BF0
:105070001E491F4C98684A68637A821ADB039A4279
:1050800002D34860FEF716FDFFF71EF9FFF7F2F8AE
:10509000012000F02FFD00F0E3FB2368DB0701D5C2
:1050A000FEF7BAFF0820C4E71024214206D00D4BBA
:1050B0001B78002BD5D1FEF7FDFDD2E7012421425C
:1050C00007D0104800F06CF806F092FA00F0F8FCF7
:1050D000C7E70424080020402142ABD0FEF7C0FE01
:1050E000BFE7C046EE63FF1FDC61FF1FC061FF1F0B
:1050F000D061FF1F1942FF1FCC61FF1FB461FF1F6A
:10510000EC61FF1FFC41FF1FF0B51B4B1B4F1B88C1
:105110003A8804001A4E1B4D85B09A420DD8328849
:105120009A420AD3184B1A882B889A4205D1174AFB
:10513000174B12881B889A421BD0052001F008FAF1
:105140003B8802AA13803388019053802B88114D2D
:1051500093800F4B02A91B88D3800F4B2A781888A5
:1051600002F024FF0D4B08212878019A1C7006F0EC
:105170002FFA05B0F0BDC046BA63FF1F0E42FF1FF5
:105180000C42FF1F0A42FF1FB863FF1FB663FF1FD9
:105190000842FF1F1664FF1F1042FF1FB463FF1F6A
:1051A00013B50C4B1C78002C11D1002801D00A4BF0
:1051B00018600A4A0A4B11780A4A10780A4A019282
:1051C0000A4A0092002205F095FA200016BD11242B
:1051D000FBE7C0461564FF1FB063FF1F1464FF1F89
:1051E0000464FF1F1664FF1FF063FF1FF463FF1FBB
:1051F00010B5064B12201B78052B06D1044B132249
:105200001988044B187801F07FFB10BD1564FF1F4F
:105210001042FF1F1664FF1F10B500240122114B1E
:1052200052421870104B1C70104B1A8002F018F983
:1052300004220F4B21001A700E480C3206F0C0FAFF
:10524000102221000C4806F0BBFA07220B4B1C6011
:105250000B4B1C700B4B1C700B4B1A700B4B1C70C8
:1052600010BDC0461664FF1F1564FF1F1042FF1FCC
:105270001464FF1F0464FF1FF463FF1FF063FF1F2C
:10528000CA63FF1FC963FF1F1242FF1FC863FF1FCE
:10529000F8B5174C0600257806A814240078052DCB
:1052A00023D1B41F134FA5B21824BD421DD88D1FA2
:1052B000ADB2BD4219D8FA256D00AA4215D21D0023
:1052C0000D4F0A3DADB2BD420FD80C4C26800C4CA0
:1052D00021800C4900240A800B4A1380FFF714FF39
:1052E0000A4B0421187806F06BFC2000F8BDC0467C
:1052F0001564FF1F790C0000750C00000E42FF1FA3
:105300000C42FF1F0A42FF1F0842FF1F1664FF1FC7
:10531000F0B50BB20D0089B0002B00DB70E1A44E9C
:10532000307806F0CDFB041E50D00378A22B00D1BC
:1053300022E1D02B1AD0912B45D143780E2B42D1AC
:105340009C4B82889A423ED19B4A83681278052AF8
:1053500039D1032018567F2835D0984B1B68002B75
:1053600031D05B68002B2ED098472CE0807807283E
:1053700029D806F08DF90428183F3F74A8D863781F
:10538000002B0CD101218C4B19708D4B1A78002AFF
:105390005BD08C4B307801F0C9FE002855D0072235
:1053A000854B1A7051E061780029F8D1E378002B21
:1053B00011D0854A854B1278307801F0B7FE6070C5
:1053C0006378002BEBD1200006F002FC8020000265
:1053D000684009B0F0BD784B1B78022BF3D0012157
:1053E000307806F02DFB0028EAD10121307806F054
:1053F000BFFBE5E76378002BD1D16F4F032807D1BE
:105400003B78052B02D101333B701EE00223FBE702
:105410006F4B1A886F4B0293002A0BD01B78002B1E
:1054200003D00121307806F0D3F83B78062B04D165
:10543000013BE9E7029B1A70F7E7042B41D10121F8
:10544000029B3078197006F093FB5C4B1B68002BB5
:10545000B9D01B68002BB6D0574A107884E7637820
:10546000554F002B27D10622211D5B4806F000F97D
:1054700062895A4B5A491A80A2895A4B1A80E38989
:105480000B800521397058490A80584A1380228AB6
:10549000574B1A80574B1B78012B09D11F2001F065
:1054A00057F8FA22920042430421307806F090F82F
:1054B0000022484B75E7312B00D070E70022454BA6
:1054C0001A700323A0E706220021434806F078F96A
:1054D0000023454A04211380444A30781380444A0B
:1054E000138006F06DFB0821307806F069FBA37984
:1054F000083B5A425341304A03331370304B1B78F8
:10550000002B06D0334B30781A78002A06D001F0F1
:105510004BFE0122314B52421A8096E7012119704D
:1055200006F026FBF5E70821307806F049FB6378A2
:10553000002B00D047E72C4B2D4F0293E388029AB3
:1055400004211380294B307803932389039A138015
:1055500063893B8006F074FA002800D033E7264BBD
:105560001B68002B00D12EE7039902983A8809881E
:1055700000881B68984726E74379132B00D022E761
:105580000389012B0AD11D4B1B78022B06D1082160
:10559000307806F015FBFFF72BFE14E7052000F02E
:1055A000D7FF08210200307806F012F80BE7C0465A
:1055B0001664FF1F051400001564FF1FB063FF1F72
:1055C0003842FF1F1942FF1FEA63FF1FCB63FF1F13
:1055D000EC63FF1FEE63FF1FBD63FF1F1042FF1F41
:1055E000C463FF1FC663FF1FBA63FF1FB863FF1FBB
:1055F000B663FF1FBC63FF1FAC63FF1FB463FF1FD5
:105600008020C001014200D0E2E6CB0731D5324B09
:105610001B78002B1DD0314E05AC3378052B1AD1E9
:10562000023B23702E4B21001B7823722D4B1B78DD
:1056300063722D4B187801F01DFD002809D007205A
:105640002A4B30701B68002B03D01B68002B00D046
:1056500098470120BCE60E20254B06221B782549E1
:105660002370254B1B78637002ABC01806F000F85E
:10567000D8E7022308001840194209D0174B1B78BD
:10568000052B03D11D4B188805F0C2FF02209FE6B1
:105690000424214203D0FFF737FD200098E60823B9
:1056A00008001840194200D193E6154B1C78012CD4
:1056B00003D0022C0DD008208AE6124B124A13495F
:1056C00013481B881288098800880094FFF7E0FDC2
:1056D000F1E7FFF78DFDEEE7EE63FF1F1564FF1F97
:1056E0001242FF1FC863FF1F1664FF1FB063FF1F36
:1056F000CA63FF1F1342FF1FC963FF1F1042FF1F32
:10570000B463FF1F0842FF1F0A42FF1F0C42FF1F26
:105710000E42FF1F10B502A804880B20002C10D1E8
:10572000496808784978090201430C48814209D147
:10573000022119800A4B59881170DB7800205BB276
:10574000537010BD074C0A20A142FAD102211980E2
:10575000034B998811705B79F0E7C0466E2A000010
:10576000B461FF1F6F2A0000F7B5150008AA16885C
:105770004A680F4F14785278120222430A24BA4220
:1057800014D10122DBB2019200962A0005F0B8FE86
:10579000041E0BD1074B1B68002B07D068782A78B2
:1057A0000002104342425041013098472000FEBDA4
:1057B000022900002864FF1F30B501250379040089
:1057C000BFB02B4225D01449408805F005FA284285
:1057D0000CD0124B01A95B8D00220B8002234B8061
:1057E0000F4B5B888B80608802F0D6FA0D49608889
:1057F00005F0F2F9C0070CD50B4B01A91B8800225C
:105800000B8002234B80064B9B888B80608802F0C4
:10581000C3FA3FB030BDC0462064FF1F3C42FF1FAB
:10582000B461FF1F1864FF1F9642FF1F10B5074C9D
:105830000749200005F086F92000064905F082F9A5
:105840000721054A054805F03FF910BDFFFF00009C
:105850002064FF1F1864FF1F68BD00113C42FF1F3A
:1058600010B5024803F01AF910BDC046B95700112F
:1058700070B55F25082607498400CA788B784001F7
:105880002A40B3433440A843234302438B70CA7079
:1058900070BDC046AD42FF1F010043B204205A0054
:1058A00002409B000C3003401A43152310B5044CF2
:1058B000E0789843143B0B4018430243E27010BD5C
:1058C000AD42FF1F10B5054B082419790A00A24309
:1058D000002801D022000A431A7110BDAD42FF1FFB
:1058E00010B5054B4024D9780A00A243002801D006
:1058F00022000A43DA7010BDAD42FF1F0821F8B53F
:10590000324D334BAE7804000E40AE70984204DD49
:1059100067232B70473B6B70F8BD2E4B984203DA20
:10592000E0232B703A3BF6E700232B706B7083B2B9
:105930001A0029485F3292B2284F82422CD9002C9B
:1059400003DA5B421CB204232B70053420B20A2117
:1059500005F046FE04B2FA239B009C4232DB08238A
:105960002A7813432B706421200005F039FE0A21A8
:1059700000B205F085FE09B22A787B5C13432B70D8
:105980000A21200005F02CFE0A2100B205F078FE65
:1059900009B27B5C6A780AE06970002CDBDA5B4252
:1059A0001CB204232B70F3226B78092CE8DC134320
:1059B0006B700A21200005F063FE09B27B5C1E4378
:1059C000AE70A9E7632CCEDCEDE7C046AD42FF1F09
:1059D0001B4E00001DFCFFFF2A08000092BD0011B5
:1059E0000823F7B5194FCD003E7904001E403E71E3
:1059F000EDB2632806DD5F3333433B7120231D4343
:105A00007D71F7BD0300093305DA20235B42334380
:105A10003B71A623F3E70E4B019300280BDA042316
:105A2000444224B23B710A21200005F029FE019B6B
:105A300009B25B5CE3E70928F5DD0A2105F0D0FD3A
:105A4000019B00B21B5C1E433E71ECE7AD42FF1FA1
:105A500092BD0011F8B50A4F05003B780E00002BEF
:105A60000CD0084C2000FEF743FC33002A00200035
:105A70003978FEF731FD2000FEF778FCF8BDC0460E
:105A80003364FF1FB442FF1F70B50A4E0A4D062251
:105A90003100280006F024F8002809D0074C310016
:105AA0000622280005F0E4FD07212000FFF7D2FFC1
:105AB00070BDC046AD42FF1F2D64FF1F2C64FF1F49
:105AC000E622402110B50A4B1A70403A5A703E3215
:105AD0009A70DA780A40DA70082219791140053A8A
:105AE0000A431A7147225A71FFF7CEFF10BDC04614
:105AF000AD42FF1F10B500282AD0164C0A21022300
:105B0000E05E05F06DFD00B2FFF7F8FE0423E05EF5
:105B1000642105F065FD012100B2FFF761FF237AE2
:105B20000024132220009A426041C0B2FFF7D8FE41
:105B30000320FFF79DFE2000FFF7AEFE064B18780E
:105B4000053843425841C0B2FFF7BCFEFFF79CFF47
:105B500010BDC046B461FF1F1564FF1F70B500255E
:105B60000A4C2000A571FEF7C3FB10233E21200044
:105B7000074AFEF7B1FCA84200D13E35054B200094
:105B80001D70FEF7F3FB0123A37170BDB442FF1F2C
:105B900082BD00113364FF1F0200F0B501270A48DF
:105BA0000A4E51188B1A002B00DCF0BD0824157822
:105BB0004308684038404000805B013C58406D0815
:105BC000002CF5D10132EDE7FFFF0000A2BD00116E
:105BD000F0B500250F269D4200DBF0BD4C5D0709A6
:105BE00044403440A400A05801357840F3E7000059
:105BF000F0B589B06A460D000B000F271100103573
:105C00001C780133260024093E401670547002327D
:105C1000AB42F5D12023024AFFF7DAFF09B0F0BD0D
:105C2000A8BD0011F0B54E780B7889B036020C0093
:105C3000170001901E43012A61D9954B9E4200D85E
:105C400077E001339E421CD1062A17D1CA788B789F
:105C500012021A430B791B0413434A7912061A43A2
:105C60008C4B5A6100221A705A808B4A5A608B4AB8
:105C70009A608B4ADA60002009B0F0BD8822520594
:105C8000EEE7884B9E423CD182498B78002B00D0B6
:105C9000F6E00C2A31D10F22A3789343E278120266
:105CA00013432279120413436279120613434B60A3
:105CB000E279A07912020243207A00041043627A4A
:105CC00012060243CA60E27AA07A120202437648C0
:105CD0004A81834208D804236E49142201980B702C
:105CE00005F0C6FC1420C7E71201D21889235B0512
:105CF0009A42F0D801238B70BDE7022AFAD005231F
:105D0000EAE76A4A01239642E6D1FFF771FA052FC6
:105D10000CD9E378A2781B021343227912041A43A8
:105D200063791B061343624A0393136005F0A8FED0
:105D3000A1E7584D2B78002B9DD1AB78002B00D1DB
:105D4000A0E02B8901339BB20093B34200D091E0D5
:105D5000132AD4D9CF7C8B7C3F02122120001F4311
:105D6000FFF71AFF874200D08EE0002E3DD1E37886
:105D7000A2781B0213432279E96812041A4363795B
:105D80001B06134303930A228B4212D1FF23A370F5
:105D9000E370237163716B89002B09D1E37B227C53
:105DA0001B0212041343A27B13431B0901336B81B3
:105DB00000226B89002B8ED0002A67D168683701DA
:105DC0003818000B6B6900030390984205D968618D
:105DD00005F0D6FEEB780133EB7068681022A11C49
:105DE000381805F0FDFD2E8145E76F89009A7B1E6E
:105DF0009BB293423AD1E278A37812021A432379F4
:105E000005A81B04134362796C6812061A43EB68F9
:105E100000920392211D0C22049305F029FC01201D
:105E2000260004A940421036FFF7E2FE013F012F91
:105E300017D1009A0B232861824200D04CE704223C
:105E40001C49200005F0CCFD042203A9686805F078
:105E500067FEE968039AFF23914200D13CE7F73BD4
:105E60003AE73100FFF7C4FE1036DFE70923B742F7
:105E7000A4D831E7009BB34200D9FCE607232BE707
:105E8000022329E7032327E7062325E70A2323E73D
:105E9000FFFE0000BC42FF1F00000111FFFF0000D9
:105EA0005048593601FF0000FFFF001102FF0000BB
:105EB00034F00040C842FF1F10B5034C0B00012214
:105EC000210000F06BFA10BD796000110B8870B5ED
:105ED00006000D000224162B11D92B0003220949BC
:105EE00000F05CFA041E0AD1074B2A881B88191C93
:105EF000934200D9111C300089B200F0EFFA200063
:105F000070BDC046A56000115A64FF1F10B54A78E5
:105F10000400013A0B000220012A07D80A78002A5F
:105F200004D005222000024900F038FA10BDC04616
:105F3000D36000110A7810B50B0004000220002A7B
:105F400004D007222000024900F028FA10BDC04604
:105F50007F6100110A7810B50B0004000220002AAE
:105F600004D009222000024900F018FA10BDC046F2
:105F7000E561001110B5034C0B000B22210000F06D
:105F80000DFA10BD1562001110B5034C0B000D2267
:105F9000210000F003FA10BD8762001110B5034C18
:105FA0000B000F22210000F0F9F910BDE162001191
:105FB0000A7810B50B0004000220002A04D0112238
:105FC0002000024900F0EAF910BDC046F16200115C
:105FD000002310B51322190000F0E0F910BD0000F5
:105FE00010B5034C0B001722210000F0D7F910BDAB
:105FF00043630011002310B51922190000F0CEF9F7
:1060000010BD000010B5034C0B001B22210000F056
:10601000C5F910BD7D630011F7B584890D00060038
:106020000121002C22D000238268D3561778002B40
:106030001EDA0C2C1AD90C3CA4B213194088009318
:10604000230002F086FE431E984101307B06DB0FE1
:106050006B703F23013C1F40A4B22870AF70AC802E
:10606000002C07D0B3680133AB6000210800FEBDEF
:106070000020EBE7AC60F8E70B7803704B884370C7
:106080004B881B0A83700B79C3700420704704206F
:10609000022B06D10020537811781B02009A0B4383
:1060A000138070470B8803700B881B0A4370022013
:1060B00070470420009983420AD1537810781B025C
:1060C00003430B80D37890781B02034300204B805E
:1060D0007047F8B50D004B7801240021461C037071
:1060E0002B788B4201D82000F8BD6B78B01C4F1C78
:1060F000012B10D1890069184B88022233704B881C
:10610000B9001B0A7370691805F022FD04360434C7
:10611000A4B2F9B2E4E7122359436B185A88043148
:1061200032705B8810221B0A7370691805F010FD2D
:1061300012361234ECE770B5049D14001E00052BD6
:1061400001D8042070BD637812781B0213432B80A2
:10615000E378A2781B02134302226B802A71211D6F
:10616000681D063E05F0F4FCB2B22A81E92AE8D89F
:106170002800A11D0A3005F0EBFC0020E2E7002317
:1061800010B50A789A4201D8900010BD9A008A187A
:106190005488013304705488DBB2240A4470948814
:1061A00084709288120AC2700430EAE710B51100B8
:1061B000029C062B04D004201022142B01D010BD09
:1061C000022222714B7808781B0203432380CB788C
:1061D00088781B02034363800431601D05F0B8FC1E
:1061E0000020ECE710B50C788B7804315C43E4B206
:1061F00003702200013005F0ABFC601C10BD0420D0
:10620000022B06D10020537811781B02009A0B4311
:106210001380704710B50C000A88023105F098FC15
:10622000208810BD70B504000D0004981100012BEA
:1062300001D8042070BD16785278120232430280D1
:106240000200F13255701470E125002C00D10C359C
:10625000023B9AB24280AA42EBD80231043005F0E8
:1062600077FC0020E6E70420009983420AD15378A6
:1062700010781B0203430B80D37890781B020343F2
:1062800000204B80704710B50C000A88023105F0E1
:106290005FFC208810BD000070B501211E000420A5
:1062A000049C0E400B4218D1CB40DDB28D4214D974
:1062B0000A49DBB2098899420FD32300EE331D70DF
:1062C0003300580011184978165C09023143013334
:1062D0002152D9B28D42F4D8002070BDD442FF1FA4
:1062E00010B50C000A88023105F032FC208810BD80
:1062F00010B50C788B7804315C43E4B20370220053
:10630000013005F025FC601C10BD10B5110002988D
:10631000032B01D8042010BD14785278043B1202DC
:1063200022430280CA788C781202224342809AB2B9
:106330008280EB2AEED80431063005F009FC0020FB
:10634000E9E710B50C000B8803700B881B0A43703B
:106350004B8883704B881B0AC3708A8804300631CF
:1063600005F0F6FBA088043080B210BD0420012B9C
:1063700003D100201378009A1370704710B50C00F9
:106380000B8803700B881B0A43704A880230043163
:1063900005F0DEFB6088023080B210BDF0B589B038
:1063A00003931E4B029242000700D05A019102F063
:1063B00020F81325061E2DD0029B01240370019B9B
:1063C000002B04D0001903999847001984B26B463A
:1063D0001B7A5BB2002B0FDA1021380002F01CFB95
:1063E0001925002813D130003219E1B202F066FC01
:1063F000051E0CD10C34A4B2042304AA380005A94C
:1064000093800696948101F0AFFD051E02D0300006
:1064100005F0B6FA280009B0F0BDC0465864FF1F69
:1064200070B505000C0000280CD00020814209D076
:1064300010222000044905F08BFB01202B782373E8
:106440006B78637370BDC046E8BD0011F0B50600FF
:106450000D0017001C0085B002291BD00020102958
:1064600007D1022B07D0102B03D115E00020102CF0
:1064700008D005B0F0BD69463800FFF7D1FF2A000B
:1064800069460BE069463000FFF7CAFF2200694603
:10649000380004E0022BE9D12A003900300005F071
:1064A0003FF9E6E7031CF02800D9F0230320084950
:1064B0009AB2013A0B80D317034006499B189B10F0
:1064C0000B80D30F04499B185B100B807047C046AC
:1064D000D842FF1FD642FF1FD442FF1F034B1B8829
:1064E0008B4202D3024B4000C1527047D842FF1F7B
:1064F0005864FF1F014B4000185A70475864FF1F33
:106500001722014B1A8070475864FF1F70B50500B1
:106510000E2005F01DF9041E13D0D02303700023B4
:106520000622837007494570033005F011FB064BC6
:106530002100DA8A62811B7E2373044B187805F0F0
:10654000F7F870BD7464FF1F6464FF1F2843FF1FCA
:10655000262803D8024B4000C05A70470148FCE788
:10656000DA42FF1FFFFF000070B506000C00094D66
:106570001C220021280005F023F9074B1E70074B51
:106580001C7005F0B5F90123002801D0002312206A
:106590002B7070BD6464FF1F2843FF1F8564FF1FBD
:1065A00070B505000D4C0800E260A16010220021CA
:1065B000656005F04DF9012803D11021A06802F0B3
:1065C00058FD10220021280005F042F9012803D1CE
:1065D0001021606802F04DFD70BDC0466464FF1F6D
:1065E00070B5041E05D1002903D006220D4805F020
:1065F000AFFA0D4B1D78012D11D1002C05D10222CF
:106600001A7004F0FDFF280070BD00221A70074BBD
:106610001B78FF2BF7D02000FFF778FFF3E700256A
:10662000F1E7C0467464FF1F6464FF1F2843FF1F27
:10663000030010B5002801D1002010BD00780B4ADE
:10664000002803D15988D1821B7913761378022B45
:10665000F2D10023984200D103331370044B1B780E
:10666000FF2B01D0FFF752FF0120E6E76464FF1F14
:106670002843FF1F002911D000280CD04B79012896
:1066800003D140225242134303E03F221340032828
:1066900002D001204B7170474022F4E70800FAE76E
:1066A00070B5094D0100287800280BD0074C062250
:1066B000200005F04DFA21002878FFF7DBFF2000CD
:1066C00004F0CEFF70BDC0468464FF1F5E64FF1FF0
:1066D00000290AD0012808D13F224B799343C02BCF
:1066E00003D0403B5A425341981C704770B5174D38
:1066F00006002B78FF2B15D00A2005F029F8041E80
:1067000010D0D0230370C83B8370114B11491B7804
:106710004670C3700622043005F01AFA210028786A
:1067200005F006F80C4B1B78012B0DD10B4B1B68A9
:10673000002B03D09B68002B00D09847084B042106
:106740001878084A05F0DCF970BDC0462843FF1FE1
:106750008464FF1F5E64FF1F8064FF1FAC64FF1F23
:10676000B064FF1F60EA0000014B98687047C046A4
:106770006464FF1F014BDB68186870476464FF1F87
:10678000074B10B5DA68136801331360054B1878AE
:10679000FF2803D08021C90105F0EAF910BDC046E9
:1067A0006464FF1F2843FF1FF7B50E0002F0C8F80E
:1067B000051E1CD00E4B06621F78002F00D10778F3
:1067C000AB791020019304F0C3FF041E0FD0D02337
:1067D0000380C73B8370019BE91DC3700622043010
:1067E00005F0B6F921003800E66004F0A1FFF7BD1E
:1067F0002643FF1F014B18787047C0468464FF1F73
:10680000054B002805D1054B1A78054B002A00D10D
:10681000014B18007047C0467464FF1F8464FF1F5B
:106820005E64FF1F014B58687047C0466464FF1FD9
:10683000024B1868431E9841C0B270478864FF1F1E
:10684000421E03000120152A03D9FF3B5A4253413F
:10685000D8B27047F0B51C0000230E0085B003903D
:1068600002920B70029A934201D3002019E0E55C7A
:106870005A1CD2B2002DF8D0029851198142F4DC92
:106880000233DFB2A35C18000193FFF7D9FF0028A1
:1068900007D0013D019A0399EBB233708A4202D1CD
:1068A000E01905B0F0BDDB19DBB2DBE710B50C0079
:1068B00002F09EF803001220002B03D0210058881C
:1068C00004F0DEFF10BD000070B50E4D840063596A
:1068D000002B15D0186A002801D005F011F82B59AB
:1068E000586A002801D005F00BF82B59986A002847
:1068F00001D005F005F8285905F002F800232B51C6
:1069000070BDC0469464FF1F1C4B70B504000E00A0
:10691000150099420AD11A4B1B68002B01D1122095
:1069200070BD1B68002BFAD09847F9E7154B9942C8
:1069300015D1134B1B68002B0AD01B68002B07D006
:106940009847002804D1104B1C70104B1D70E7E7CE
:1069500029002000FFF7AAFF0028E1D1F3E7080093
:1069600001F0EEFF0028DAD003780320A342D7D14C
:106970002900300004F084FFD2E7C046FEFF00008B
:106980009064FF1FFFFF00008D64FF1F8C64FF1FDA
:10699000F7B50400808801F0D3FF0025A84203D09A
:1069A0000578A08802F008F81C4E3378002B1FD021
:1069B000AB421DD11A4B28001978FFF777FF00284A
:1069C00018D000233370A3790820A778A6880193F4
:1069D00004F0BEFE011E0DD0D0230370CA3B8370AD
:1069E000019B477086808371280004F0A1FE01E0BE
:1069F000002DE8D1A0880B4B8200D358002B01D08A
:106A0000FFF762FF1721A088FFF768FDA08801F05B
:106A100027FDA08801F0FEFDF7BDC0468D64FF1F75
:106A20008C64FF1F9464FF1FF0B587B01D000CAB92
:106A30001B88070001930DAB1B88142002930EAB3B
:106A40001B88160003930FAB1B880091049310ABB7
:106A50001B88059304F07CFE041E1AD0D02303701B
:106A6000CB3B47708370C670062229000430002D8E
:106A700011D005F06DF8019B21006381029B009805
:106A8000A381039BE381049B2382059BA37404F0F1
:106A90004FFE07B0F0BD04F093FEECE7F7B50093AE
:106AA00008AB1B8807000C200D001600019304F0B2
:106AB0004FFE041E13D0280001F042FF00280FD023
:106AC0000078D0232370C93BA370009B2100238151
:106AD000019B6770A580E680638104F029FEF7BD05
:106AE000014B1878EDE7C0462843FF1F13B504009B
:106AF00064890389C2888188C0780094FFF7CEFF3B
:106B000013BD000010B5044C2068002803D004F029
:106B1000F7FE0023236010BD9864FF1FA122F0B58B
:106B2000818892004A43384B384F1B6804009B18F9
:106B30009D2292009B18827989B01A603B68002BD5
:106B40005FD01D78324B1B68002B04D05B68002B94
:106B500001D000209847260008363100E079FFF781
:106B6000B7FD237DE0710200E0780493638A290079
:106B70000393238A0293E3890193A388009333004C
:106B8000FFF752FFE378002B0BD1E289A379A188AC
:106B900002920196E27928000092012201F0DAFEC9
:106BA000E0703B68002B20D0FFF7ACFF194D287830
:106BB00000281AD0184B1978FFF778FE002814D057
:106BC0002B78E67808200793A78804F0C1FD011E02
:106BD00009D0D0230370CA3B4670837087808671CA
:106BE000079804F0A5FD00232B701721A088FFF75C
:106BF00075FCA08801F034FCA08801F00BFD09B001
:106C0000F0BD064B9DE7C0463409FF1F9864FF1F87
:106C1000AC64FF1F8D64FF1F8C64FF1F2843FF1FA0
:106C2000F8B5070008000E0001F08AFE041E18D017
:106C30002620FFF78DFC051E00D12578062004F0E4
:106C400087FD041E0DD00021062204F0B9FDD023DB
:106C50002370C23B21006770A370A680E8B204F0E5
:106C600067FDF8BDF0B585B001930AAB1B7807004E
:106C700002930BAB1B7808000D000092039301F008
:106C80005FFE061E22D0102004F062FD041E1DD0FF
:106C90001022002104F094FD2620FFF759FC002863
:106CA00000D13078D0232370C13BA370009B21001A
:106CB0002372019B67706372029BA580A372039B82
:106CC000C0B2E3720C9BE36004F032FD05B0F0BD8E
:106CD000F7B50D00019001F033FE071E20D00E2005
:106CE00004F036FD041E1BD02620FFF731FC061EE3
:106CF00000D13E78D0232380C53B0622A370F91D26
:106D0000E01C04F025FF019B2A0063810123DD4084
:106D10001A401D40210022736573F0B204F008FD93
:106D2000F7BD0000F0B585B0029010000D0017000F
:106D30000A9E039301F004FE041E31D0029B002B37
:106D40002ED1039B02795B0724D51223134304221F
:106D5000002E08D10B99002905D10C99002902D1E8
:106D60000D9900291AD01A430D9B2271002B00D0D7
:106D7000C9E0002E00D1CFE0002D00D0CCE0606A49
:106D8000002801D004F0BCFD1C21300004F0B0FE4E
:106D9000606205E002239A430E33D7E793432371E1
:106DA000654BBA00D458002C00D1AAE0002E10D0B8
:106DB000236A002B03D11C2004F02AFD20625E4BC5
:106DC000BA00D358186A002803D01C22310004F0FE
:106DD000BFFE0C9B002B12D0574CBB001D596B6A99
:106DE000002B03D1162004F013FD6862BB00E358AA
:106DF000586A002803D016220C9904F0A9FE0D9BB6
:106E0000002B11D04C4DBC006659B36A002B03D146
:106E1000142004F0FDFCB0622B59986A002803D0BE
:106E200014220D9904F094FE380001F089FD051E2E
:106E300067D0414BBA00D358002B62D01A6A342075
:106E4000002A00D11C389A6A002A01D0143080B27E
:106E50000B9A002A01D01C3080B25B6A002B01D053
:106E6000163080B204F074FC041E4AD018220021AF
:106E700004F0A6FC2620FFF76BFB0190002801D14F
:106E80002B780193D0232370029B200063700A2388
:106E9000294EA370039BBD00A371AB59A780196A4B
:106EA0001830002905D01C22A06004F051FE2000FB
:106EB00034307359996A002907D00300142214331F
:106EC000E060029304F044FE02980B9B002B08D074
:106ED00003001C221C330B992061029304F038FE3E
:106EE00002987359596A002903D01622606104F090
:106EF0002FFE6B462100187904F01AFC3800FFF7CA
:106F0000E3FC05B0F0BD10220D9B0D991B69A01884
:106F1000236204F01DFE2CE70B9B002B00D13FE702
:106F2000012D00D03CE7606A002801D004F0E8FCA5
:106F30001C210B982AE7C0469464FF1F10B5044C2F
:106F40002068002803D004F0DBFC0023236010BD80
:106F50008864FF1F0B4B07B51A68002A01D1002077
:106F60000EBD6946531C012012780731FFF772FCF1
:106F70000028F4D002780123100018401A42EED005
:106F8000EEE7C046A464FF1FF0B51F4F01203B6829
:106F900087B0002B25D09B78059300F0B3FB002829
:106FA00021D00A20FFF7D4FA04000B20FFF7D0FA13
:106FB000164B05001E78731E9E413B68F6B2191DE4
:106FC000D878FFF757FB3B682900DA7A043303923D
:106FD0009A7901930292009033002000059A04F000
:106FE00027FD07B0F0BDFFF7B5FF002805D006204C
:106FF000FFF7AEFA04000720D8E70820FFF7A8FA49
:1070000004000920D2E7C0468864FF1F8464FF1F84
:1070100070B50A4E040033780D00FF2B0DD004200C
:1070200004F096FB011E08D0D0230370CE3B4570C0
:107030008370C470307804F07BFB70BD3843FF1F51
:1070400070B5040006200D0004F082FB011E0AD07A
:10705000D0230370CD3B8370054B44701B68858043
:10706000187804F065FB002C01D0FFF767FF70BDB6
:107070008864FF1FF8B5264F06003B680D001124F9
:10708000002B05D10522234B1B78134202D1122479
:107090002000F8BD204A10241268002AF8D0127887
:1070A000002AF5D0DB0719D52B789A1E012A1AD8A9
:1070B0000C2004F0ADFB132438600028E8D0002336
:1070C0000A22437029000670023004F041FDFFF7E8
:1070D0005BFF041E0AD0FFF731FFD9E700F012FB77
:1070E0000028E1D1E4E7002BE2D0D0E70B4B1B787E
:1070F000032BCDD11D20FFF72BFA094B1880002858
:10710000C6D0084B04211878074A04F0F9FCBFE701
:107110008864FF1F8564FF1FA464FF1F8464FF1F32
:107120008264FF1FB064FF1F60EA0000F7B501939F
:10713000194B14001A78052306000F0012201A427A
:1071400021D0012920D1154B1D68002D1BD0022014
:107150001F2C18D8002C02D0019B002B13D0104BF1
:107160001F221E706E1C0021300004F029FB0199C3
:107170002200300004F0ECFC310020002C70002FC5
:1071800006D004F03DFBFEBD064B12201D68DCE777
:1071900004F0F6FAF7E7C0468564FF1FA464FF1FFA
:1071A0003843FF1FA064FF1FF8B50F4E1224336849
:1071B000002B17D01B780F3C834213D100250B4FB7
:1071C0000221387804F0FCFC094B042138781D803A
:1071D00004F0F6FC074B28001D8033685C7004F057
:1071E000A7FC04002000F8BD8864FF1FB064FF1FE7
:1071F0009C64FF1F8264FF1F70B5012823D11B4CC4
:107200002388002B03D01A4A1578002D07D0194B7C
:107210001B68002B02D01878FFF7C6FF70BD3B2B10
:1072200002D93C3B2380F9E7134E0221307804F069
:10723000C7FCFA222388920002215A43307804F0D6
:10724000C7F92580EAE70B4B1B68002BE6D00B4BF8
:107250001B785B07E2D5084B0221187804F0B0FCDC
:107260000022024B1A80FFF769FED7E79C64FF1FDC
:107270008064FF1F8864FF1FB064FF1F8564FF1FC9
:10728000F8B51E4D2868002803D004F039FB002310
:107290002B601B4E3068002803D004F031FB002324
:1072A0003360184F05243B7818002040234221D03A
:1072B000154800F02BFA3B78234213D0202004F02D
:1072C000A7FA2860002813D02022002104F078FAC1
:1072D000202004F09DFA041E306005D020220021F9
:1072E00004F06EFA002004E0286804F009FB2C602A
:1072F0001320F8BD00F00AFAF4E7C046A464FF1FAB
:10730000A064FF1F8564FF1F2C43FF1F10B50A4CAC
:1073100023681A1E0ED0002808D10130587004F0DE
:1073200007FC002805D02368002B02D00021FFF7BE
:1073300087FE0122100010BD8864FF1FF7B5274E9D
:10734000050033680191181E21D05C78244F012C70
:1073500030D1FFF7FFFD002825D02000FFF7F8F817
:107360000400412814D91F4B022118781E4A04F04A
:10737000C7FB1E4B3C3C1C80022233685A703B7892
:10738000002B14D128000199FFF75AFE0120FEBD01
:10739000FA2292004243002AEED0124B02211878C2
:1073A00004F016F9E8E7FFF7D3F80200F3E700234B
:1073B0003B70EBE73B78002BE8D1032004F0C8F9E1
:1073C000011E08D0D0230370CC3B45708370336816
:1073D000187804F0ADF9FFF7B1FDD7E78864FF1F17
:1073E0008064FF1FB064FF1F60EA00009C64FF1F01
:1073F00010B51749838802008B4220D011D8154957
:107400008B4217D0144900205B1899B2012907D884
:10741000926811785A425341D8B2FFF7F9FD012022
:1074200010BD0E4A00209B1807229BB29A42404191
:10743000C0B2F5E783681878FFF768FFF0E7836864
:1074400099785A78090218781143FFF777FFE7E730
:107450000A20000006200000F8DFFFFFAFDFFFFF7B
:10746000014B18707047C0463943FF1F10B5064CDA
:10747000207001F041FA207804F012FB05212078F9
:1074800000F062FD10BDC046B064FF1F0BB273B5C3
:107490000D00002B00DBC4E0884B187804F010FBD3
:1074A000041E0ED00378912B0FD0A22B00D1A1E0A7
:1074B000834B1878FF2852D0210004F039F90028B6
:1074C0004DD180200002684076BD43780F2B76D0E6
:1074D00013D8052B70D00E2BEAD18088794B9842B7
:1074E0002BD8794B98421BD8784B9842E0D1A368AF
:1074F0001878591CFFF774F838E03E2BD8D1837800
:10750000032B74D06CD8012B6ED0022BD0D1704BD2
:107510001B68002B23D05B68002B20D098471EE00F
:107520006C4BC0180C28C3D804F082F91DC2C215D8
:107530000BC20B0B0B3223C23C00674BC018072851
:10754000B6D8664B1B68002B09D01B68002B06D0F1
:10755000200098470AE0A3681878FFF7C7F82000D2
:1075600004F036FBADE7A068FFF762F800289FD073
:10757000F5E7A3681B78002BF1D0554B1B68002B57
:10758000EDD01B68002BEAD0210055489847EDE765
:107590004F4B1B68002BE2D01B68002BDFD0210073
:1075A0005048F3E7504B1B68002BD8D05B68002B8A
:1075B000D5D021004348E9E7FFF7EAF9CFE7808813
:1075C0004A4B984203D04A4B984200D070E7464B52
:1075D0001B68002BC3D05B68002BC0D02100D5E70F
:1075E000153B012BBBD963E7FFF798FAB7E7FFF725
:1075F0007DFAB4E73F4B1B78042B07D100236A4682
:1076000013800179408800F0C5FCA8E7364B1B6861
:10761000002BA4D05B68002BA1D00100364898470E
:107620009DE7012421420AD0294B1B68002B04D07E
:107630005B68002B01D000209847012043E78B07AF
:107640000AD5264B1B68002B04D05B68002B01D0A9
:1076500020009847022036E70421280008400D4208
:1076600000D131E7254E3388002B21D0013B9BB25E
:107670003380002B1AD1FFF7DBF800280AD0204B0B
:107680001C70164B1B68002B04D05B68002B01D0CC
:1076900020009847FFF7C6F8694601F001FD6846EB
:1076A000FEF7FEFF1D20FEF753FF308004200AE79F
:1076B000024B187804F084FAF8E7C046B064FF1F64
:1076C0003943FF1F0E2000000120000009100000B8
:1076D000A864FF1FFEDFFFFFAFDFFFFFAC64FF1FEB
:1076E0000C2000000B2000009064FF1F0D20000004
:1076F000132000008564FF1FFFFF00008264FF1F4E
:107700008064FF1F10B501F09BF910BD014B18609C
:107710007047C046AC64FF1F0B880020162B01D8B1
:1077200017230420014A13807047C0465A64FF1F84
:1077300000207047074A03001188814207D09188D2
:107740000020994202D101308000101870470020BB
:10775000FAE7C046B864FF1FF0B58F7806000D0049
:10776000C5B01E2F15D1FFF7E5FF051E03D100247C
:10777000200045B0F0BD00223B003100C0780092EF
:1077800000F0B2FB0400A81C00F0D2FBFF23EB705A
:10779000EEE7264B062403931B78FF2BE8D0182F27
:1077A000E6D87B08224A013BDB0002929A589446B5
:1077B000002ADDD0029AD3185B68002BD8D0087855
:1077C000002802D14B78012B02D10624122FCFD1F1
:1077D00007AFAB88697800976446AA68A047041E83
:1077E000C6D1AB78029A5B08013BDB00D3183900A5
:1077F00030005B689847041E0BD1AB78042BB6D0E1
:10780000039A310010782200009700F06DFB04000D
:10781000AEE76A78002AABD1AA7805A93B8808713F
:1078200030000A704B80FEF747FBA0E73C43FF1F88
:10783000F8BD00111D4B37B5050098420BD000294B
:107840000AD1FFF777FF002805D11948FFF772FF2B
:10785000002800D0058037BD01291AD1FFF76AFF43
:10786000041EF8D001235B420380A378FF2BF2D0E3
:10787000FE2B07D00023E0781422009329001E334A
:1078800000F032FBA01C00F053FB01235B4263803D
:10789000E1E70229DFD1013901F0BEF80028DAD191
:1078A0002800FFF747FF041EDFD1D4E7FEFF0000EA
:1078B000FFFF0000022210B5074B52421A80074812
:1078C00001325A809A80DA8000F07EFA044801F092
:1078D00025F8002010BDC046B864FF1F597700117D
:1078E000357800110388F7B50400002B02D102257A
:1078F0002800FEBD42680221137825485268FEF731
:10790000A5FD00282ED0234F01253A88002AEFD06C
:10791000802321885B0201259B1A9942E8DC0C2018
:1079200003F076FF061E31D03B8822889C46002358
:107930001800019561469DB2491989B2AA421BD827
:10794000002801D062443A8000233000082208C099
:10795000210004F0FDF8104A1368002B13D1002514
:107960001660C5E76268022113780C485268FEF77A
:107970006DFD0028C7D1BAE760681D01401941813B
:1079800001330198D6E71A001B68E6E71325AFE735
:1079900066BE00113A43FF1FB464FF1F64BE0011AE
:1079A000014B18707047C0463C43FF1F14230A0068
:1079B00010B51A40194204D00122102101F048F8F4
:1079C00010BD4B06F9D4012088434000F8E710B5FC
:1079D00014008B0604D50122102101F039F810BDE6
:1079E00008230A001A40194202D14BB2002B0FDAC9
:1079F000102101F02DF8002808D02300F2331B7865
:107A0000002BECD0F1342378012BE8D10020E6E7FD
:107A100003208907FAD4E2E7F0B51F00184B85B0C0
:107A20001C68019002910392002C27D1200005B020
:107A3000F0BDA5683301ED186B89019A934211D30B
:107A4000029A93420ED8002F04D10A9B002B10D12A
:107A50002C00EBE73B002978039A6868FEF7F6FCF8
:107A60000028F2D10136B6B2A388B342E1D8246827
:107A7000DAE7A3680A9A5B891380E9E70026F3E74F
:107A8000B464FF1F37B50C000A884988012391426E
:107A900017D3002A15D0651D23792A0002210A4830
:107AA000FEF7D4FC102300280BD0237961882088AE
:107AB00000242A000094FFF7AFFF0A23A04200D061
:107AC000230018003EBDC04666BE001113B50A0073
:107AD00008884988012388420BD8002809D000244F
:107AE000137905320094FFF797FF0A23A04200D0D4
:107AF0002300180016BD13B50A0008884988012321
:107B000088420BD8002809D000241379053200944C
:107B1000FFF782FF0A23A04200D02300180016BD01
:107B2000F0B58BB003904A8808880E00012382428A
:107B300055D3002853D00023012704AC2370002222
:107B4000718813000092FFF767FF051E3ED0207872
:107B5000002835D12B78022B18D167706A898300F1
:107B60000130E31880005A8069680222201803F06F
:107B7000EFFF23780133DBB22370042B19D93B00CC
:107B80006889013080B2002BD9D01FE002236370D6
:107B9000122358436A89231804305A8069681022D6
:107BA000201803F0D5FF23780133DBB22370002BBC
:107BB000E5D10C4A6B899B185A425341DBB2DFE78F
:107BC0006378012BE4D12B78022BC7D022780A23CB
:107BD000002A04D021000398FEF798F9002318002A
:107BE0000BB0F0BD0100FFFF0F4BF0B504001868AB
:107BF000002816D083685D89A54207D88288AE1810
:107C0000B44203DA12019A18934201D10068EFE7F7
:107C10001E005F891036A74204D1002900D00D80D4
:107C20001800F0BD3300EFE7B464FF1F70B5050026
:107C30000C0008880021FFF7D7FF03000120002B6C
:107C400004D022002800197AFFF7C1FE70BDF7B5F5
:107C50000C00002501902300EE331B78AB4201D8C5
:107C600000200AE06B00E65A00213000E718FFF719
:107C7000BBFF002802D126800130FEBD017A0198A9
:107C8000FFF794FE002802D03B882380F5E70135FA
:107C9000EDB2E0E710B5040008880021FFF7A4FF6B
:107CA00003000120002B03D02000197AFFF77EFE8D
:107CB00010BD0000054B1B68002B01D1180004E02B
:107CC0009A6852898242F6D198887047B464FF1F3F
:107CD000F0B50E27002687B0039302ABFF183E8055
:107CE00005001F4B40891400984207D02B780130C3
:107CF00000976A6880B2FFF78FFE060002212B789A
:107D000018486A68FEF7A2FB00280FD06C89200093
:107D1000FFF7D0FF002802D0013C0419A4B2039B56
:107D2000002B00D01C80300007B0F0BD02212B7862
:107D30000D486A68FEF78AFB0028E7D102212B78FC
:107D40000A486A68FEF782FB002807D0002EDED0C2
:107D50003B88A342DBD17489013CDFE76C89DEE715
:107D6000FFFF000066BE001164BE001162BE00117C
:107D700010B50C00FFF7DEFC03000220002B0AD038
:107D8000002C00D023609B781720FE2B03D00138F5
:107D9000FF2B00D1002010BD73B50D0001A9040018
:107DA0001600FFF7E5FF172805D0002E04D12900A3
:107DB0002000FEF727F976BD01221021200000F0F7
:107DC00047FE0028F3D0F6E7014B18607047C04625
:107DD000C464FF1F37B56B469D1D010004000222DD
:107DE000280003F045FC2B88B02B0ED12379122BF1
:107DF00009D12300FA331B78012B06D101216088B9
:107E000000F0E0F801E01B2BF8D037BD10B5054BB2
:107E10000421187000F098F8FFF74CFDFEF770FB96
:107E200010BDC046C864FF1F0020F0B50BB20F00A4
:107E300087B0834234DA274B187803F041FE051EE1
:107E40002BD00378A02B25D103AE3100FEF7E4F848
:107E5000041E0BD1B378DB0724D51F4B06341B68F7
:107E6000002B03D03100688898470400A8680028D8
:107E700001D003F085FD002C08D1184A039B134064
:107E8000174A934206D0B3781B2B03D00121688890
:107E900000F098F8280003F09BFE80200002784054
:107EA00007B0F0BD0F4B1B68002B10D03100688865
:107EB0009847041EDAD07378002BD7D1B27801A985
:107EC0000A704B800C716888FDF7F6FFCEE7062438
:107ED000F1E7C046C864FF1FC064FF1F00FFFF003A
:107EE00000011200C464FF1FF7B50190FC200D00D3
:107EF00017001E0003F02CFC04001320002C12D0ED
:107F0000B02320002370089BF422677065802671DF
:107F10000830002B08D0190003F01AFE2100019848
:107F200003F006FC0020FEBD089903F049FCF5E7CC
:107F300010B5041E06D00078FD2803D803F050FCCD
:107F4000FF23237010BD00000A1F93B210B5040078
:107F50000220032B05D882400020024BD1529B18EF
:107F60009C7010BDE864FF1F0B8870B5043B0400D3
:107F70000D000220032B0BD80121200000F04CFD46
:107F800003001420002B03D02900200000F0DEFBAA
:107F900070BD000007B51300034A00920A000121DA
:107FA00000F02CFC0EBDC046D181001107B5019236
:107FB00003220092024B0A00122100F049FC0EBD80
:107FC0004F82001107B56B4601AA11800449D88081
:107FD00008780633012802D1190003F039FB07BDE8
:107FE000C964FF1F0C4B10B518700023FF210B4A0A
:107FF0001380138193819380094A538013705172C7
:1080000093819372D174D3821375517703F040FD3D
:1080100000F0FCF910BDC046F864FF1FE864FF1FC4
:10802000CA64FF1FF0B58DB06B46002003910C228F
:108030009B5E834200DBB0E05D4B187803F040FDAF
:10804000051E00D1A4E00378902B00D09DE006AF80
:1080500001004688380000F013FA7968040000290E
:1080600000D19CE03B88052B6ED13B89032B1CD9AA
:1080700005AC200000F0A2F86288172A61D839897F
:10808000131D994231D17968237804310291D907BF
:1080900038D5607800F08EF9071E06D000230371F2
:1080A0002378012B08D0132B23D0A868002800D1F7
:1080B00078E003F065FC75E06288029909A800F099
:1080C000A6F80290380000F08BF909AA2378387AD4
:1080D0000192002231000092029A00F012F9380059
:1080E00000F064F9029B002BDFD0300000F080F933
:1080F000DBE70378032BD8D16288029909A800F046
:10810000D6F8DEE7122B13D1029909A800F0B5F8D2
:10811000021EEAD127498B88002BC6D0887909A98D
:108120002378019161780091310000F0EAF8BCE712
:10813000002302AA93833000617809AAFFF72AFF7F
:10814000B3E71D4B0993F6E7042B02D09A1F012ACF
:10815000ABD8184A043B9B00995A0029A5D0D218E5
:10816000907831003A0000F0AEF800289DD13B88AD
:10817000042B03D001213000FFF724FF012C04D190
:10818000A868002801D003F0FBFB280003F020FDC5
:108190008020039B0002434018000DB0F0BD012871
:1081A00000D182E701213000FFF70CFFEDE7C04668
:1081B000F864FF1FE864FF1F010017000B780370CD
:1081C0004B784370CB788A781B0213434380704707
:1081D0000A88030002700A88120A42700A88012A7B
:1081E00006D14A8882704A88120AC27004207047F9
:1081F00002208242FBD14A8804309A704A88120ACF
:10820000DA708A881A718A88120A5A71EFE710B5F3
:108210000400012082420CD94B780A781B021343D8
:108220002380834206D1CB788A781B021343638074
:10823000002010BD022BFBD1CB788A781B021343A0
:1082400063804B790A791B021343A380F0E70B8804
:1082500003700B881B0A43704B8883704B881B0A82
:10826000C3708B8803718B881B0A4371CB88837121
:10827000CB881B0AC3710820704703000120082A1D
:1082800014D14A780878120202431A80CA78887892
:10829000120202435A804A790879120202439A80F4
:1082A000CA798879120202430020DA80704710B53B
:1082B00004000120022A05D100204B780A781B0215
:1082C0001343238010BDF8B5060010200F001500E1
:1082D00003F03EFA04000120002C0ED0A0230C2253
:1082E000290023806780201D002D07D003F030FC7B
:1082F0002100300003F01CFA0020F8BD03F060FA02
:10830000F6E7F7B51E00009008AB142017001D78A3
:10831000019103F01DFA041E12D0A2230370019BE9
:1083200047704380099B057146710C220830002B71
:1083300007D0190003F00CFC2100009803F0F8F9B5
:10834000F7BD099903F03CFAF6E737B5041E0FD0E4
:108350004388002B0CD00025C1881323007A1722F4
:1083600001950095FFF7CDFFFF23658063722570AF
:1083700037BD000010B50C4904004A88002A09D016
:108380008B89002B05D00020CB8A0222834201D0AA
:1083900010BD012213000A20434300204032C8547C
:1083A000C81842800472F3E7CA64FF1F00234380A9
:1083B00003707047094B00211A0010B55C88002C2F
:1083C00006D01C79844203D10A234B43D01810BD38
:1083D00001310A330329F1D10020F8E7CA64FF1FF5
:1083E00010B50400407A03F0FBF9FF23637210BD5F
:1083F0007047043010B580B203F0FAFB002803D0B8
:108400000421494203F0CCFA10BD000070B50025EC
:10841000104CA0682580A581A580A84202D003F059
:10842000AFFAA56000250C4C0C4B606D1D8023003D
:1084300058331D70A84202D003F0A2FA65650025EA
:108440006068002801D003F09BFA013508340A2D3A
:10845000F6D170BD9065FF1F3465FF1F8465FF1F57
:1084600070B5041E09D1054D2880A881A880A86890
:10847000002802D003F084FAAC6070BD9065FF1F45
:10848000F0B54B8885B00193002343600A7905005D
:108490000F00022A00D07BE0CA88032A17D98B6814
:1084A0005E7819783602DC78D8790E4399781B7A91
:1084B00024021B020C43034353495BBA0B80331D58
:1084C00093421ED1042C04D0631F022B0ED901202D
:1084D00015E0019A4D4B1201D35A002B06D001989A
:1084E000FFF7BEFF4A4A1369013313610421B868DC
:1084F0002E812C80494203F053FA6860002005B0B9
:10850000F0BD434D042C06D0631F022B0FD9EB683E
:108510000133EB60DBE7019A3C4B1201D35A002B8D
:1085200005D00198FFF79CFF2B6901332B61374B76
:1085300030000293019B029A1B01019300230199D1
:108540008C468B52130063449C8003939E81FFF7FB
:1085500050FF039B041E986016D00421B86849425E
:1085600003F01EFAFA880100043A200003F0F0FA42
:108570000199029AFB888A5A043B9B18029A8B52F3
:108580002B6801332B60A2E7AB690133AB619EE737
:108590001E4B0293019B1E01029BF35A002B2DD010
:1085A00002998C19A068002828D0012A26D1FA88BF
:1085B0009B189BB27352A189994217D39B1AC0187A
:1085C000B96803F0C5FA029BA289F35A934200D01E
:1085D0007DE700222B81A3882B80A3686B60029B20
:1085E000F2520B4A53680133536070E7084A9368AC
:1085F000013393600198FFF733FF68E7044A53693A
:1086000001335361F6E7C046FA64FF1F9065FF1F10
:108610000065FF1F70B5051E15D10B4C0B4B188064
:10862000230058331870606D002802D003F0A8F9B9
:108630006565250050356068002801D003F0A0F979
:108640000834AC42F7D170BD3465FF1F8465FF1F4D
:10865000F0B51700A12285B0920001934243394B37
:1086600006001B680C009B18D933FF331D78FDF7FB
:1086700041FF0430854204DD3000FDF73BFF04304C
:10868000C5B2BD4207D33A0000213000019B03F080
:108690002FF805B0F0BD2900380003F0E1F9230000
:1086A000C6B250331E700393019B290063653800E6
:1086B00003F09EF8CBB20293002B02D0039B01364D
:1086C0001E7000262300503303931B78B34204D856
:1086D000606D002831D10020DBE7029A2800002AD3
:1086E00004D0013B1000B34200D02800F700E71986
:1086F000387002F0F5FF786000280ED03A780199C2
:1087000003F026FA019A3B780136D3180E4A0193FA
:10871000D369F6B20133D361D4E7039B1870606567
:10872000A74205D1084A1320D36A0133D362B0E7C8
:10873000606803F025F90834F2E703F021F900231B
:108740006365C8E73409FF1F0065FF1FF7B50D001B
:1087500007000421686803F023F92B8904000370E3
:108760002B891B0A43702B8883702B881B0AC370CC
:108770002E8902250436F6B2F42E15D81B4B9F42E3
:1087800014D10C2002F0E4FF1135011E0CD090230F
:1087900003708E3B0371043B4380154B8460C6809D
:1087A000187802F0C5FF00252800FEBD5C237B433E
:1087B000104AD3180093583301931B78002B0FD124
:1087C0000300320038000099FFF742FF019B0500CB
:1087D0001B78002BE8D13800009903F081F8E3E71B
:1087E000054A0725536A01335362DDE7FEFF0000A7
:1087F000F864FF1F3465FF1F0065FF1FF0B587B0E9
:10880000009017200F0016000193FFF7F2FD1325CB
:10881000041E19D00C98031E02D00199201D984700
:10882000030AE370052302AAA07004309081277028
:108830000098667003A993800494FFF787FF051ED4
:1088400002D0200003F09CF8280007B0F0BD000023
:10885000F0B587B01F000CAB1B7803910593012185
:108860000DAB06001C78049200F0D6F81425002801
:1088700021D02000FFF77EFD0135041E1BD01149D9
:10888000059B0A7803700132D2B2131EC68001D153
:1088900001231A000B7022713000049B039900978A
:1088A000FFF7ACFF051E09D1230021000648074A47
:1088B000093303F0A5F8280007B0F0BD002363805A
:1088C0002370F8E7FC64FF1F4B8300113075000034
:1088D000F8B505000E00064C064F2368002B02D0A9
:1088E0003100280098470434BC42F6D1F8BDC04698
:1088F000A065FF1FB465FF1F0123064A5B4253803A
:10890000002313715362044A136053609360D36071
:1089100013617047B465FF1FA065FF1F02000023AD
:1089200010B506499C000859002801D1625010BDBD
:108930000133052BF6D11320F9E7C046A065FF1FD0
:10894000034A5388181A4342584140421040704726
:10895000B465FF1FF0B585B002930AAB1F780CAB6E
:108960001B88009008000E0001920393FFF7E8FFB8
:1089700005001120002D1BD10E48FFF7E1FF040078
:108980001520002C14D006220B99A771E01D03F0CE
:10899000DFF8019B30002371029B29006371009B6B
:1089A00066802370039B6562E381FFF791FF2800D7
:1089B00005B0F0BDFFFF000010B5FFF7C1FF0400D8
:1089C0000220002C12D060880121FFF781FF606A2D
:1089D000002801D002F094FF28220021200002F09C
:1089E000EFFE012300205B426380207110BD000078
:1089F00030B5074A074C5588010013780020A5427E
:108A000004D05B1A59424B415842104030BDC04619
:108A1000B465FF1FFFFF0000084A10B501230C00DA
:108A2000904208D0FFF78CFF031E04D00379234047
:108A30005A1E9341DBB2180010BDC046FEFF000075
:108A4000024B1879431E9841C0B27047B465FF1FAE
:108A500070B504000D001600FFF772FF002804D166
:108A60000D4B9C4200D0143070BD416A0379052043
:108A7000002907D012221A40102A02D10520002E08
:108A8000F2D10F20DB06EFD5897E0C20A942894167
:108A9000494249420840E7E7FEFF0000030010B5E5
:108AA000002800D110BD0348034A41889142F9D003
:108AB0009847F7E7B465FF1FFFFF0000002330B5BC
:108AC000C45CCD5C6C40D4540133102BF8D130BD64
:108AD0000F23002210B5C45C64002243CA54C25C58
:108AE000D209013BF7D210BD0200010010B52032BF
:108AF000103102F0D5FE10BDF0B58BB00390102000
:108B000005931700049102F083FE0090102002F0FC
:108B10007FFE009B13240190002B05D000280CD170
:108B20001324009802F0ECFE019B002B02D01800E9
:108B300002F0E6FE20000BB0F0BD102002F068FE4F
:108B40000600102002F064FE13240500002E00D160
:108B5000AEE0002819D01022002102F031FE3200D0
:108B60002900039802F09CFE041E0ED133787F2B5F
:108B700051D830000099FFF7ABFF009B1B787F2B8B
:108B800053D801990098FFF7A3FF300002F0B8FE18
:108B9000002D02D0280002F0B3FE002CC1D110201D
:108BA00002F036FE0600102002F032FE0290002E87
:108BB0007CD0002878D03A000F3223000125121112
:108BC00005D00F333B4015B25A4253411BB26A1EC7
:108BD0001201002B33D0049BD2B298180099029A4C
:108BE000FFF76CFF013D10220021300002F0E8FD8C
:108BF000ADB2049F2D017D19AF4242D0002C33D07D
:108C0000300002F07DFE029B002B00D189E71800A6
:108C100002F076FE85E729003000FFF759FF2800B3
:108C20002549009AFFF74AFFA7E729000098FFF7B8
:108C30004FFF28002049019AFFF740FFA5E70F21C9
:108C40000F4004998A18D9B28F4208D9D15C06A87E
:108C500019540133102BF6D1029A0199C0E7791A01
:108C600048424141C901F2E73900300006AAFFF746
:108C700025FF3200039806A902F012FE1037040007
:108C8000BAE7002CBCD13000029906AAFFF716FF04
:108C9000320006A9039802F003FE08220400310006
:108CA000059802F055FFABE71324A9E71324AAE7C0
:108CB000002800D06EE733E76CBE0011F0B58BB032
:108CC0000F0016000225009000283FD0002A3DD05A
:108CD0000B1DDBB21800029302F09AFD1135041E41
:108CE00034D0FDF747FD05003A000099201D02F041
:108CF0001FFEEBB20393E3702B0CDBB22F0A009341
:108D00006370FFB22B0E2370A7700193FDF72CFD4B
:108D10001022010006A802F00BFE2100029A04AB0B
:108D200006A8FFF7E9FE051E0DD1039B082233704C
:108D3000009B04A9B370019B7770F370301D02F0A3
:108D4000F7FDFDF71DFD200002F0DAFD28000BB055
:108D5000F0BDF0B58FB00D00149E03900492059302
:108D6000002A03D1022420000FB0F0BD002EF9D05C
:108D70000398FFF7E5FD1424071EF4D072783378CA
:108D800012021A43B3781B041343F27812061A43F3
:108D9000036A0192934201D30133E3D1002D03D042
:108DA0003B7901249B07DED50822002106A802F0AA
:108DB00007FD059B13240433DBB21800029302F075
:108DC00027FD051ECFD0059A0499043002F0B0FDAE
:108DD00004223100280002F0ABFD390010221031CE
:108DE0000AA802F0A5FD2900029A06AB0AA8FFF71F
:108DF00083FE041E0FD1082206A908A802F098FDE0
:108E00000822311D08A802F08BFC012807D1019926
:108E10000398FDF7C9FC280002F072FDA3E70124C6
:108E2000F9E7000070B51C4C05002368181E10D02F
:108E3000002D14D11A78002A0CD1981C083202F0A7
:108E400087FE02F035FC0135002808D123681D702B
:108E5000012070BD0A331800082202F079FE236851
:108E6000002BF5D0122002F073FC061E0DD0C1239A
:108E700021680370457002311022023002F068FE52
:108E800023683100587802F053FC206802F038FD66
:108E900000232360DCE7C046DC65FF1FF8B5040053
:108EA0002020FDF755FB0D4EA700BB590500002BF8
:108EB0000DD000280BD0D878FF2809D108492A0006
:108EC0000C55F35907480333611802F099FDF8BDBA
:108ED000290002F09DFD0028F0D1F8E7F865FF1F9A
:108EE000E065FF1FF5A0001170B5064D84006359C1
:108EF000002B05D0D87802F073FCFF226359DA709A
:108F000070BDC046F865FF1F70B506008CB00C0040
:108F1000150000213022684602F052FC3100102278
:108F2000684602F005FD1D2021000322684402F07E
:108F3000FFFC6846FFF7D8FD2D210400032228001E
:108F4000694402F0F5FC20000CB070BDF0B50700DC
:108F5000160097B001931CAB1D7830221EAB009118
:108F60000AA800211C7802F02BFC102239000AA864
:108F700002F0DEFC1022002102A802F021FC0722F0
:108F8000310002A802F0D4FC072202AB9818631E3D
:108F90009C41019902F0CCFC02AB9C732B005A1E41
:108FA000934102AAD3730021102206A802F008FC04
:108FB00006221D9907A802F0BBFC1A2002ABC018BC
:108FC00006221F9902F0B4FC102200990EA802F0AC
:108FD000AFFC102202AB0EA908781C78013A604061
:108FE000D2B2087001330131002AF5D10AA8FFF787
:108FF0007BFD102212A904000EA802F0A9FD102288
:1090000006AB0EA908781D78013A6840D2B2087004
:1090100001330131002AF5D10AA8FFF765FD0443A9
:1090200010222098E4B212A902F082FC200017B0AE
:10903000F0BD70B50E0014008CB00100102268461F
:109040001D0002F075FC3100082204A802F070FC3B
:109050002100082206A802F06BFC6846FFF744FDD9
:1090600004001022280008A902F062FC20000CB0C5
:1090700070BDF8B506000D0000243719AC4200D3CE
:10908000F8BD02F095FC030A3B70631CDBB20137AC
:109090009D4203D90234F054E4B2EEE71C00EDE740
:1090A00073B506000C000225002819D0002917D03E
:1090B000032101A8FFF7DDFF6B469A793F231A4091
:1090C000013313436A463000937101A92200FFF770
:1090D0001BFF051E04D10322E01C01A902F038FD8C
:1090E000280076BD03785807DA08C00FD200800048
:1090F0009B0710439B0F1843C0B2704707230B40D8
:10910000C908C9000B4303707047000070B5040024
:10911000FFF7EAFE134DA4006359002B21D0186A13
:10912000002801D002F0ECFB2B59986E002801D0EA
:1091300002F0E6FB2B59D86E002801D002F0E0FBCC
:109140002B59186F002801D002F0DAFB2B59586F09
:10915000002801D002F0D4FB285902F0D1FB0023F3
:109160002B5170BDF865FF1F0E4B8000C35870B5C2
:109170000C00002B0FD09D68002D0CD02B78201DEB
:109180000B706B784B70A97CFFF7B8FF2B7E2372B6
:109190006B69E36070BD10220021200002F010FB1B
:1091A000F8E7C046F865FF1F014B18607047C046DE
:1091B000F465FF1F074A03008000825810B5002A9B
:1091C00006D0D088984203D1012901D1FFF79EFF34
:1091D00010BDC046F865FF1FF0B5264E95B087005C
:1091E0000B93BB590500099112200A92002B31D034
:1091F000D888FFF7A5FB04001420002C2AD02800F3
:1092000010A9FFF7B1FFBB591E781D6A002E23D0AD
:109210000895FDF7EFFA07000020FDF7F1FA079037
:10922000A379E61D069310AD0CA9089800F0E2FAA8
:109230000EA9280000F0D7FA0B9B0A990493069B0D
:1092400009980293079B0396019300970EAB0CAA13
:10925000FFF77CFE15B0F0BDFDF7CCFA06903000AC
:10926000FDF7CEFAE31DA779079310AB060008932C
:10927000DAE7C046F865FF1F30B50C4C85002A5967
:10928000030085B00120002A0ED018006946FFF7C0
:109290006BFF2B591A78D888054B002A00D1054B53
:1092A0006A46072100F0D9FB05B030BDF865FF1F05
:1092B000E7970011F597001130B5094C8500295941
:1092C00085B010226846253102F042FC2A5911214E
:1092D000044BD0886A4600F0C0FB05B030BDC046E4
:1092E000F865FF1F9198001130B5094C8500295988
:1092F00085B010226846353102F02AFC2A59112126
:10930000044BD0886A4600F0A8FB05B030BDC046CB
:10931000F865FF1FCF980011F7B54D4F860010205C
:10932000F4590D0002F074FAF3592062186A1322FE
:1093300000286CD0033A29009C6802F009FCF3591C
:109340001A780192002A58D11E6A227D317B9446F8
:1093500051400122019F114201D167461740217DF2
:10936000914339432175377B4F40BC466046002707
:10937000800701D44F081740012102208F40227D31
:1093800082433A432275377B5740BC4660460027EC
:10939000400701D497080F400420227DBF0082437C
:1093A0003A432275627D002794466046727B4240B4
:1093B0000A4201D167460F400121627D8A433A4348
:1093C0006275777B5740BC4660460027800701D412
:1093D00057080F400220627D7F0082431743677564
:1093E000767B00227E40760701D4BA080A40042624
:1093F000617D9200B1430A4362756A78002A08D001
:109400006278002A05D005220533DA7700221000A1
:10941000FEBD04222979114205D1A17C114202D15D
:109420000533033AF1E7019A21782C78002A02D11A
:109430000A002100140018220429E8D8042CE6D8D8
:1094400005206043034A05331218525CDDE7C0462D
:10945000F865FF1F7CBE001110B50A001121024BF8
:1094600000F0FBFA10BDC0462B9900110B0030B57F
:1094700087B001AD2B806B4604001100981D0822B7
:1094800002F066FB2A000B212000024B00F0E5FAF7
:1094900007B030BD5399001110B50A001121024BDD
:1094A00000F0DBFA10BDC046A799001113B50B0000
:1094B00011006A4613706B4604000622581C02F025
:1094C00047FB6A4608212000014B00F0C6FA13BD95
:1094D000C799001110B50A001121024B00F0BDFA26
:1094E00010BDC046179A00117FB505000B4BAA00AE
:1094F000D4580800002C0FD0666F237FE2882178B3
:109500000396266F0296E66E0196A46E0094FDF710
:1095100009FC2800FFF7FAFD7FBDC046F865FF1F74
:1095200010B51721FFF7E0FF10BD000070B50A006D
:109530000D00064B0221040000F08FFA0600297886
:109540002000FFF7D1FF300070BDC046F798001132
:1095500070B586B000236A461370836804001D78D6
:10956000681E0A2859D801A902F092F80606333776
:109570003B3F43474B4F5300180000F042F906238E
:1095800012284BD000281BD16088FFF7D9F9082397
:10959000002813D04279002A47D1264B1A78072396
:1095A00012070BD5244B1A680723002A06D0166829
:1095B000002E03D0290001AAB04703006A461370A9
:1095C0006B461B786088002B2AD1FFF767FC06B03A
:1095D00070BD180000F06CF9D4E7180000F087F9AE
:1095E000D0E7180000F093F9CCE7180000F0ADF9CF
:1095F000C8E7180000F0C3F9C4E7180000F0F6F956
:10960000C0E7180000F0F6F9BCE7180000F013FA04
:10961000B8E7180000F013FAB4E707236A4613709E
:1096200069466088FFF782FFD1E70523012AC5D18B
:10963000024BB8E78564FF1FF065FF1FF465FF1F4D
:10964000F8B52C4F8600F35904000D00002B40D0D4
:10965000DA8882423DD15A78062A33D11A78002A14
:109660002ED0012099681A6A097D014206D0157B27
:10967000054203D007225A700120F8BD02200142A2
:1096800004D0157B054201D00922F4E704200142F1
:1096900004D0127B024201D00B22ECE7164B1B6870
:1096A000002BE9D05B68002BE6D020009847BB591F
:1096B00000215B78122BDFD12000FFF715FFDBE7DD
:1096C0000E4BECE7112A04D1002900D032252900E5
:1096D000F2E7002D08D12000FFF732F9002803D06F
:1096E000102302791343037121002800FDF798FA33
:1096F000C2E7C046F865FF1FF065FF1FF465FF1F56
:1097000070B50E4E8500AB590400002B13D01B78AA
:10971000002B11D10A4B1B68002B04D05B68002B77
:1097200001D02000984773595B78122B03D1002198
:109730002000FFF7D9FE70BD024BECE7F865FF1F74
:10974000F465FF1FF065FF1F094B8000C358102010
:10975000002B0CD01A6A002A09D09B68002B06D077
:10976000127A1B7E101C9A4200D9181CC0B2704796
:10977000F865FF1F70B503000D0014000220002AD9
:1097800030D000292ED013700B78081D53704B7801
:109790009370FFF7A7FCE070012002212B7A237160
:1097A0006B7B034063716A7B0A401343042263713D
:1097B0006E7B1640334363716E7BF608F6003343CD
:1097C00063712B7B0340A371287B014000200B4376
:1097D000A371297B0A401343A3712A7BD208D200CC
:1097E0001343A37170BD10B50A0001000120FFF7FB
:1097F000C1FF10BD10B50A0001000220FFF7BAFF3B
:1098000010BD70B506000C000220002E30D00029DB
:109810002ED07378201D0B70B3784B70F178FFF762
:109820006DFC01223579257271794B1008001340C7
:10983000934010400343881010408000C908034340
:10984000C9000B436373B1794B1008001340934078
:1098500010400343881002409200C9081343C90016
:109860000B4321202373FCF773FE854201D21220A3
:1098700070BD2220257AFCF76BFE8542F7D823784D
:109880001820042BF4D86378012BF1D80020EFE7DF
:10989000030010B50220002909D0002B07D00322B5
:1098A000481C0A7019000D3202F052F9002010BD58
:1098B00003000222080010B5002B06D0002904D0B6
:1098C0000E32591C02F044F90022100010BD0300B2
:1098D00010B50220002909D0002B07D00422481C13
:1098E0000A7019000C3202F033F9002010BD10B5D7
:1098F000FFF7DEFF10BD03000220002906D0002B79
:1099000004D0052200200A701B784B7070470300BA
:109910000220002B08D0002906D05B7800200B70B5
:10992000013B082B00D918307047030010B5022006
:10993000002909D0002B07D00622481C0A70190004
:109940000A3202F005F9002010BD10B5FFF7B0FF94
:1099500010BD02000B00022010B500290ED0002A15
:109960000CD007211970118859701188090A997053
:1099700011180822D81C02F0EBF8002010BD0300DB
:109980000A00022010B5002B0CD000290AD09978CB
:109990005878090201431180901CD91C082202F05A
:1099A000D7F8002010BD030010B50220002909D00F
:1099B000002B07D00822481C0A701900921802F0E8
:1099C000C7F8002010BD02000B00022010B50029CE
:1099D0000BD0002A09D00921197011781818597074
:1099E000511C062202F0B4F8002010BD10B5FFF79C
:1099F0005FFF10BD02000B00022010B5002A09D045
:109A0000002907D05178197011180622581C02F04D
:109A10009FF8002010BD030010B50220002909D0D6
:109A2000002B07D00A22481C0A701900063202F0E7
:109A30008FF8002010BD10B5FFF73AFF10BD0200EF
:109A40000B00022010B5002A06D0002904D018000F
:109A50005178FFF753FB002010BDF0B585B017001B
:109A60001E006A4606230500080091819380FEF7D8
:109A7000C0FC1324011E02900CD03800B047041E15
:109A800005D1280001A9FEF76FFA041E02D0029842
:109A900001F076FF2800FFF701FA200005B0F0BDC5
:109AA000F0B504008BB0019115000021102202A82E
:109AB00001F086FE334EA700B85900283CD0C38879
:109AC000A34239D10378002B36D14278062A18D127
:109AD00002000100553235310C3006ABFFF7A9FA10
:109AE000002829D12000FFF72FFE020006A902A8B6
:109AF00002F02EF8200002A901F052FE01200BB066
:109B0000F0BD816E002917D00B8A112A28D19D4201
:109B10000ED101981231093A01F002FE012807D155
:109B2000BB5920009D6EFFF70FFE29000200DEE703
:109B300032212000FFF7D8FC2000FEF701FF061EAF
:109B40001BD0416A002918D00B8AAB4215D10822DC
:109B50000198123101F0E4FD01280ED1716A0AE08A
:109B60009D42E9D108220198123101F0D9FD012866
:109B7000E2D1BB59996E8A7EB9E7200002F048F81D
:109B8000BCE7C046F865FF1FF0B56B4D87007E59F6
:109B900085B0337802900393002B00D087E0B36840
:109BA000346A01937078062817D101221B7D134275
:109BB00002D0217B114218D10222134202D0217B14
:109BC000114251D10422134203D0237B134200D00F
:109BD0008BE0019B5A7DEB5991E007380428F8D8B7
:109BE00001F056FD032E42678300B36E002B03D1B4
:109BF0001C2001F00DFEB066EB599C6E002C1CD0B1
:109C000010220021200001F0DBFD0298FFF79CFDEF
:109C100001002000FFF72DFA01F0CAFE208220008B
:109C200008211230FFF725FA0298FFF78DFDA07684
:109C3000EB592100D888FFF70FFC0822EB591CE0F4
:109C4000B36E002B05D01A00198AF0881232FFF784
:109C50000DFC0222019B197DEB5911423DD0207B66
:109C600010423AD0073208E0F488FCF7DBFD01002F
:109C70002000FFF711FC0A22EB595A70029B9C004E
:109C80002A595378073B042B11D8D088FEF758FE89
:109C900000284ED0C3895A08D2182849029B02983E
:109CA000CB542B5941180433254801F0A9FE05B0C7
:109CB000F0BDFCF79FFD03000120834201D100208D
:109CC0000393EB59DE88FCF79BFD039902003000FB
:109CD000FFF7ECFB019AEB59117D042211420CD0E5
:109CE000217B114209D00B22C7E7F688FCF73CFD27
:109CF00001003000FFF7EEFB6BE7019A527D012176
:109D00000A4204D0607B084201D00C22B5E7022150
:109D10000A4204D0607B084201D00E22ADE7042144
:109D20000A4204D0627B0A4201D01022A5E7122227
:109D3000A3E7FA225200B0E7F865FF1FFC65FF1F9A
:109D4000FFA0001110B5064B1A780423100018402C
:109D50001A4200D00348FFF727FA002010BDC04682
:109D60008564FF1F4043FF1F70B50400FFF7D4FA5E
:109D7000051E43D12000FFF77FFA234EA400A0590F
:109D80008268937CDB0708D50321036A1B790B40AB
:109D9000012B02D1017F0B430377431DD97F8B1E1B
:109DA000022B0DD8022900D00121C088FCF790FFBA
:109DB000042133591A7F59700A431A77280070BD5D
:109DC00001290CD102231022437000210C3001F034
:109DD000F7FC305910213530FFF74BF9EEE7052934
:109DE000ECD10223D118437010220C3001F0B0FEE8
:109DF00004233259117F0B431377EAE7082518280B
:109E0000DCD1053DDAE7C046F865FF1FF0B58BB041
:109E1000059143887E4F9E00F45915000493002C51
:109E200015D1012902D000200BB0F0BD101D5778CC
:109E30001678FFF757F9EB68320002932B7A0499F2
:109E4000019300903B002000FCF70CFFEBE7E38858
:109E5000049A934201D00820E6E72378012B00D131
:109E6000D4E0059B581E092800D9CFE001F010FC72
:109E700005CE0A29CC506C859AB229000498FFF7C8
:109E800073FFD1E7200029001022453001F060FE69
:109E9000B9594B78042B02D1013B4B70C3E70B003F
:109EA0000A00253335320C310498FFF795F90498F0
:109EB000FFF702FA0522431E9841BB59C0005A70B1
:109EC000B2E7200029001022553001F041FE049B2A
:109ED0004F4C9D00295904980A0006AB55320C31AD
:109EE000FFF77AF929591022453106A801F018FC2C
:109EF000012808D10498FFF7F7F90590002804D14C
:109F000006222B595A7005988EE708230593FAE725
:109F100063780C2B7AD1E36E002B03D11C2001F067
:109F200077FCE066BB59D86E00286FD0102229005C
:109F300001F00EFEBB590498DC6EFFF705FC0D2204
:109F4000A076BB595A706EE7E06E00285ED0637849
:109F50000D2B5BD12B8808220382A91C123001F043
:109F6000F7FDBB599A68517D0222114226D0186A2A
:109F7000407B104222D00C32E4E763780E2B45D1AF
:109F8000236F002B03D1162001F042FC2067BB5940
:109F9000186F002803D01022290001F0D9FD0F22EC
:109FA000BB59CFE763780F2B30D1206F0622691C95
:109FB000103001F0CDFDBB599A68517D0422114249
:109FC00003D0196A497B1142D5D100210498FFF7CB
:109FD0008BFA28E7636F002B0DD0BB59586F002810
:109FE000F3D01022290001F0B3FD0122BB595242E7
:109FF0005B6F1A61E9E7142001F00AFCBB59606746
:10A000005B6F002BE9D126E72978DFE707200BE714
:10A01000F865FF1F10B5064C207001F029FD0621E0
:10A020002078FDF791FF0348FEF778FC10BDC0468D
:10A030000B66FF1FB591001100200BB270B50D002B
:10A04000834216DA264B187801F03AFD041E0DD033
:10A050000378922B0ED0A02B37D0224B1878FF28F4
:10A060003AD0210001F064FB002835D180200002A5
:10A07000684070BD43780E2B0BD03E2BEDD183781A
:10A08000052B12D0082BE8D181798088FFF7D8FA08
:10A0900008E0154B82889A42DFD183681878591CF2
:10A0A000FEF7C0FE002817D1D7E7104B1B785B07DF
:10A0B00012D50F4B1B68002B0ED09B68002B0BD0CA
:10A0C000C289811D80889847ECE7FFF741FAA068B4
:10A0D000002801D001F054FC200001F079FDC5E713
:10A0E0000B66FF1F3943FF1F182000008564FF1F08
:10A0F000F465FF1F10B50078FFF712FA10BD10B518
:10A100000078FFF7FDFA10BD0C234343084A10B551
:10A110009B185A68002A03D0012901D1904710BD2D
:10A120009B68002BFBD00029F9D19847F7E7C04680
:10A130002866FF1F01238340094A10B5946B1C4316
:10A140009463506B98435063D46B2000984301296B
:10A1500001D120001843D063116B0B43136310BD72
:10A1600000800040F0B500240127154B85B0DA6B64
:10A17000144E03921A6C0192DA64019BE3403B4255
:10A1800017D0039DE5403D400295E5B202992800B5
:10A19000FFF7BAFF316A736A002908D03900002B33
:10A1A00001D0029979402800FFF7C4FF01E0002B9D
:10A1B000F9D101340C36172CDFD105B0F0BDC04603
:10A1C000008000400C66FF1F064B01215A68C24008
:10A1D0000A4204D01B68C3401800084070471B6D3A
:10A1E000F9E7C046008000400122064B824000296A
:10A1F00003D0D9680A43DA607047D9689143D960BF
:10A20000FAE7C0460038004030B5032444430F4B02
:10A21000E25C1B199C785D7801232D1B0135AB4056
:10A22000013BA340A140DB430C00122807D808499A
:10A2300092005218116819402143116030BD054A3F
:10A2400011680B4023431360F8E7C046C3BE0011FA
:10A2500008F0004014F00040C21F70B5D4B20623CD
:10A26000092C0BD80125084C9540002908D0002165
:10A27000FFF7CAFF23682B4323600023180070BD3B
:10A280002368AB43F8E7C04600380040214BF0B5E7
:10A290001B185B78022B21D1032444431E4A1F4E16
:10A2A000A35C12199478012215008540B76B013C1C
:10A2B000E4B23D43A240B563194C122815D89B0067
:10A2C00000290CD117495B1899680A439A60012349
:10A2D000205C154A834011680B431360F0BD11499F
:10A2E0005B18996891439960F1E70E4B00290DD1F5
:10A2F00059690A435A61225C1328E8D00123203AA5
:10A3000093400A49086803430B60E7E759699143A2
:10A310005961F0E70C66FF1FC3BE001100800040CA
:10A3200008BF001100F00040A0F00040A4F0004081
:10A33000F8B500241B4E1C4D1C4B1B5D012B1FD17F
:10A34000194A9269E2401A420BD00122B256934058
:10A350002200143AD2B2022A09D815494A69134395
:10A360004B61013402360C35172CE5D1F8BD0022C3
:10A37000B2560F499200521891680B439360F0E770
:10A38000022BEED1E7B23800FFF71EFF0123584041
:10A39000C1B23800FFF77AFF3800FFF715FF687782
:10A3A000DFE7C04695BE00110C66FF1F0D66FF1F5C
:10A3B00000F00040012202388240054B002903D002
:10A3C00059690A435A617047596991435961FAE7DB
:10A3D00000380040F8B50E0001210F008740114AF7
:10A3E0000400D368FD43BB43D360831E8B4201D876
:10A3F000FFF7E0FF00212000FFF72EFF0A4A0B4B7A
:10A400005168012E05D139431B1951605E7000203F
:10A41000F8BD2940516002221C1962709A691540EA
:10A420009D61F4E700380040008000400C66FF1F8B
:10A43000012210B58240074B002906D019680A4353
:10A440001A600121FFF7C6FF10BD1968914319601A
:10A45000F7E7C046008000400C2370B50025434359
:10A460000A4A29009B181D70094B04001B185D70D7
:10A47000FFF7B0FF0123A340064928000A681A43EA
:10A480000A6005490A689A430A6070BD2866FF1F82
:10A490000C66FF1F348000403080004070B504001F
:10A4A0000E00FF2813D003250540FFF7D5FF084A0B
:10A4B000A3089B009B183F22ED00AA40AE401968FC
:10A4C00020009143314319600121FFF78DFE70BDDB
:10A4D00018380040F8B50C244443134B0500E41829
:10A4E0006368002B03D1A3681220002B1AD002222C
:10A4F00001270E4B00215B195A7028002770FFF7C7
:10A5000069FF63681E1E08D0A3683E00002B04D0BC
:10A510002800FFF759FE4640F6B228003100FFF749
:10A5200009FE0020F8BDC0462866FF1F0C66FF1F0D
:10A53000F7B5C420FF222B4B80001958002491430B
:10A540003F3A0A431A508022274F5202274E1A6080
:10A55000274B1D5D002D21D0A31E012B03D8012107
:10A56000E0B2FFF727FF012D18D11F4B9B69E34095
:10A570002B4213D0E3B218000193FFF725FE010030
:10A580000198FFF755FFE3B2143B022B1DD80121C0
:10A590007156184A8D405369AB4353613B7F002B82
:10A5A0000DD0E5B22800FFF795FF2800FFF70CFE5D
:10A5B0007B7F0100834202D02800FFF7A5FD013414
:10A5C0000C370236172CC3D1F7BD01210023715679
:10A5D000F3568D40074A9B009B189A68AA439A60DD
:10A5E000DCE7C04600E100E00C66FF1F95BE0011ED
:10A5F0000D66FF1F00F0004010B501210400FFF7B9
:10A60000E9FE0123044A002011194B70A34091690F
:10A610000B43936110BDC0460C66FF1F70B50E0062
:10A6200015000400FFF718FF0C236343094A2000BC
:10A630009B189D605E60FFF74DFFF021064B074AB7
:10A640008900051E5A5002D02000FFF705FF2800A0
:10A6500070BDC0462866FF1F0000FF1F65A10011E6
:10A6600070B5134D07202C78002C1FD198222100A3
:10A670005200280001F0FCF80123C420FF222B70B7
:10A680000C4B80001C635C630B4B1C605C600B4BD1
:10A69000195891433F3A0A431A50802252021A60D5
:10A6A0000D20074A074901F0A3F9200070BDC046FC
:10A6B0000C66FF1F00800040A0F0004000E100E0B9
:10A6C00031A5001131A30011030010B50620072B9E
:10A6D00009D8054A137001F05BF8D7210020034B1D
:10A6E000034A89005A5010BD6843FF1F0000FF1F36
:10A6F000D91AFF1F70B51D0002240C2910D8094A71
:10A70000CA40D2070CD5FBF72FFF041E08D1059ACB
:10A7100004992800FBF744FFFCF7B2FDFFF712FB9A
:10A72000200070BD1210000030B50D7802232C00FF
:10A730009C43184201D02B431C0008252300AB4347
:10A74000284201D02B00234320241D00A543204292
:10A7500001D01C4325002A230D70184204D0117823
:10A760001E3B0B43137030BD0028FCD10C21137825
:10A770008B43F7E7F8B51D0006AB1B88140007AA4A
:10A780000E000B201778002B27D10A78022A49D116
:10A790004A68507811780002244A08438018042837
:10A7A00040D800F075FF03121D1B2300F06801F074
:10A7B00037F8021CC0B2B84200D93A1CD2B220000D
:10A7C000F1682A8001F0C4F906E00222F3681B88D0
:10A7D0002A8023701B0A63700020F8BD0622EEE772
:10A7E00001232B80F3681B782370F5E7F368002BB7
:10A7F00016D008222A801A8822701A88120A6270DB
:10A800005A88A2705A88120AE2709A8822719A882D
:10A81000120A6271DA88A271DB881B0AE371DBE736
:10A820002B80D9E701202B80D7E7C04600D6FFFF59
:10A83000F7B516000A781D0008AB1F880C0001232D
:10A84000022A18D14A685078117800022B4A08432E
:10A85000801803280FD800F01BFF02254439E06858
:10A8600000F0DEFFC0B20723B84204D37B19019386
:10A87000152B02DD0D231800FEBDE0682A00310013
:10A88000C01901F065F96B4600209B88E268D0543E
:10A890001B4B1B68834203D01B68834200D0984740
:10A8A0000023E8E70B23002FE5D1022DE2D17378D6
:10A8B00032781B021343E2681380114B1B68002B94
:10A8C000EED01B68002BEBD00120E8E70B23002F14
:10A8D000D1D1062DCED12A003100E06801F038F93F
:10A8E000DEE70B23002FC6D1012DC3D1327875339B
:10A8F000012AC0D8E3681A70D2E7C04600D6FFFF2D
:10A900001868FF1F70B50C001500072837D800F035
:10A91000BFFE041436361B36242E182015290BD8FA
:10A92000184E16220021300000F04AFF22002900B4
:10A93000300001F00DF9002070BD18200229FBD174
:10A940001288114B1A80F6E718200829F4D10A0062
:10A950000E48290000F08CFEEDE718200129EBD10C
:10A960000B4B10780B49DA69FFF7DEFEE3E718209E
:10A970000129E1D1064B10780749DA6BF4E7022090
:10A98000DAE7C0460068FF1FE643FF1FDC43FF1FF6
:10A990006C43FF1F9443FF1FB443FF1F030010B518
:10A9A0000020DB0704D50721024A034800F08CF899
:10A9B00010BDC04620BF00116C43FF1F054A0300B5
:10A9C0001068002803D082889A4201D180687047BD
:10A9D0000068F6E7106AFF1F0A88030008009A4221
:10A9E00004D08A8804309A4200D0002070470000CA
:10A9F000F8B5F22200230D4F0D4E79680500424351
:10AA00003370994200D07B600A4C0021200000F096
:10AA1000D7FE00231A007C60AB4202D100203370C5
:10AA2000F8BD01332280DBB2F234F5E7086BFF1F7B
:10AA3000066BFF1F146AFF1F73B56B46019006007B
:10AA4000684615001980FCF74DFF041E11D1002D3A
:10AA50000FD07689002E11D00C2000F0D9FE0028EE
:10AA60000ED0084A0460136886808560002B02D1EE
:10AA70001060200076BD1A001B68F7E70224F8E793
:10AA80001324F6E7106AFF1F012100220A4B10B5BC
:10AA900049420A4C198099809A719A70084B20702B
:10AAA000012019805A60FFF7A3FF2078FCF778FF98
:10AAB0000448FDF733FF10BD2068FF1F106BFF1F18
:10AAC000086BFF1F75AB0011022310B5002802D0E0
:10AAD000FFF7B2FF0300180010BD0000030010B51F
:10AAE0000020DB0704D50421024A0348FFF7A4FF36
:10AAF00010BDC04634BF0011EC43FF1FF0B50E2659
:10AB000087B003930CAB1F8802ABF6180500080052
:10AB100031000292FDF768F804000120002C0FD0EC
:10AB20003088FFF74BFF03000E20002B08D05E6833
:10AB3000002E05D021002800039B029A0097B04701
:10AB400007B0F0BD0A4B10B5984207D1012200238F
:10AB500052420A808B708A808B7110BDFFF73CFFD8
:10AB60000028FAD001235B42038000238370F4E7BE
:10AB7000FFFF0000F8B5050001290AD1134E00249B
:10AB80003388F227AB4219D028001149FFF7DAFFCA
:10AB900006E0022904D10139FDF73EFF0028EDD07F
:10ABA000F8BD3B0063437268D018D35A002B09D01C
:10ABB0003A00002100F004FE0134E4B2054B1B789A
:10ABC000A342EED801235B423380DDE7086BFF1F11
:10ABD0002068FF1F066BFF1F10B5FFF7FDFE030087
:10ABE0000020834200D0987810BD0000F0B589B0F5
:10ABF0001C000EAB80CB03901E8810AB1B78049218
:10AC000002930B7A0D00DB0616D42B780593022BEA
:10AC100024D00498FFF7D2FE002812D003689C4687
:10AC2000002B0ED0029B2200019329003B006446BA
:10AC300003980096A04705E00498FFF7BFFE0028A0
:10AC400002D10E2009B0F0BD8368002BF9D00A2292
:10AC50002900039898470028D7D0F3E76B68587805
:10AC60001A786B4B000210439842D2D8043B9842AA
:10AC700010D2684B984242D015D8674BC0180128B3
:10AC8000C7D80B20002EDDD1EB681A7859683A80BE
:10AC9000200028E0614BC018032800D979E000F0BB
:10ACA000F7FC846A789E5E4B9842B2D10B20002E4E
:10ACB000C8D101233B80EB6831001B782370688981
:10ACC000013080B2FCF790FF3A88031E0ED0017865
:10ACD00002328A183A80428962704289120AA2704E
:10ACE00059680278E01C00F033FF06E004323A8035
:10ACF00031000422601C00F063FD0020A2E70B205D
:10AD0000002E9FD1EB6807A91E8804233B80330ADD
:10AD1000300026706370FCF767FF051E28D004AB77
:10AD20009A890E2304A95B183E49C668FCF7D0FF38
:10AD300000280BD12B783C486A680599FBF786FB05
:10AD4000002803D1012304AA5B42D3813278022A6E
:10AD500006D17168201D00F0FBFE3B8802333B806A
:10AD60000E2304AA9B181B88A3701B0AE370C4E778
:10AD700004ABDE81F4E70B20002E00D062E7E96827
:10AD80000398FFF729FF02233B802070000A6070C0
:10AD9000B3E70B20002E00D054E70222EB681B889B
:10ADA0003A8023701B0A6370A7E7E86800F038FD5B
:10ADB000C2B203000720B24200D243E70DD002998D
:10ADC000DBB27118994202DB921BD3B20293029B51
:10ADD000E9681A003B8089195AE70023F6E70B203F
:10ADE000002E00D02EE70722EB683A801A782270F6
:10ADF0005A7862705A88A2705A88120AE2701A79D8
:10AE00002271DA886271DB881B0AA37175E7C0467C
:10AE1000042900000228000000D8FFFFFFD6FFFF32
:10AE200003280000FFFF000064BE0011F0B58DB0E4
:10AE30006B460020089120229B5E83423DDAA64BA0
:10AE4000187800F03DFE071E32D00378B02B2CD1CD
:10AE50000079023816281FD800F01AFD17001E00CE
:10AE60001E001E0031001E0096001E001D011E0067
:10AE700052011E0073011E00CD011E0050021E0073
:10AE80001E001E008E021E00E302944B94491B8894
:10AE900078880B80FBF71AF83800FCF79BFF914B82
:10AEA0001B68002B01D038009847380000F090FE56
:10AEB0008020089B0002434018000DB0F0BDEE2238
:10AEC0000021874800F07CFC0BAA3B7B79893889FC
:10AED00000923A000D32FCF79FFD0400804B1B7876
:10AEE000002C3FD146E0804B788805937F4B410092
:10AEF000CB5A0BAE073BDBB232880293002301939F
:10AF00007B4B210006930093059BFFF76FFE744D6A
:10AF1000002810D1069B3A8A1B889A420BD1380030
:10AF20000599123000F0FCFB002804D02B786289D0
:10AF30009B00EB185A80162306A81B1832882000A5
:10AF40007989FCF7C5FE2B7804009A00AA1851886D
:10AF50000029C3D00133DBB22B70002807D006A92B
:10AF6000C98A9180634A12889A42BCD802E00121C2
:10AF700049429180002B04D059497888FAF7DAFFCA
:10AF80008AE73E890A2479E000253E89574B0693DB
:10AF90007B88069A5B009B5A033B9D4202DB002D97
:10AFA000F0D05BE0162206A812183B7B798900924C
:10AFB0003A0030000D32FCF72FFD0590002858D0E4
:10AFC0004689017A7888FCF7F1FC041E44D1464B8F
:10AFD00078880793069B4100C95A454B0439C9B28A
:10AFE00006AAD28A06930291019400930599079BC1
:10AFF000FFF7FCFD041E2FD1069B39491A88931CCC
:10B00000002D26D14B807988384B4900CB5A5119F5
:10B01000033B8B4220DD059B31485B8941190B7155
:10B02000A91C0135C9B2EDB2059145191B0A2B7156
:10B03000059B2D490433181800F08AFD2C4B059A06
:10B040001B88D318DDB22C4B9E4205D00136B6B218
:10B050009CE749889942D6D0002D0CD0204C28007E
:10B06000618800F0BDFA207021007888FAF772FF3D
:10B0700012E7059CF0E7002C00D183E77B78142BC6
:10B0800000D109E716493B794E800B700C71788826
:10B09000FAF712FF00E7162406ABE41821003889FE
:10B0A000FCF7A2FD011E00D1B7E1788822880F4C81
:10B0B00045002C5B0A4D013CE4B2029400240F4B86
:10B0C00001940095FFF792FD041E00D014E12900C1
:10B0D0007888FAF74FFFDFE6106BFF1FD842FF1F9B
:10B0E0002868FF1F1C68FF1F1C69FF1F5864FF1F93
:10B0F0000C6AFF1FD642FF1FFFFF00002A68FF1FD8
:10B10000162406ABE41821003889FCF76DFD011EFA
:10B1100000D182E178882288AE4C45002C5BAE4D90
:10B12000013CE4B202947C89AC4B01940095FFF79A
:10B130005DFD041E00D0DFE029007888FAF724FFC7
:10B14000AAE60025A44B1D803B00F6331B78A24ADB
:10B1500078880792AB4208D99E4B128806930699CD
:10B1600043005B5A013B9A4203DB0799FAF716FF4B
:10B1700092E616246B00FB18059306ABE418059BBA
:10B1800021001889FCF730FD011E03D1059B012425
:10B190001E8973E77888924B2288069C09934300A6
:10B1A0001B5B904E013BDBB20293002300960193A0
:10B1B000099BFFF71BFD041E02D0059B1E895DE75E
:10B1C0007B88069A5B009B5A079A1088328812186F
:10B1D000934202DC1B1A013B33807F4C02303288E1
:10B1E0000999001900F0B4FC2388328801359B18B6
:10B1F0002380EDB2A8E70BAA3B7B798938890092BE
:10B200003A000D32FCF708FC00250590059B002B49
:10B2100004D10A24002D00D16EE060E0059B7888FF
:10B22000197AFCF7C3FB0100041E63D1694C6C4B17
:10B23000788806940993069B4400E45A694B063CBF
:10B24000E4B20BAE32880793029401910093059902
:10B25000099BFFF7CBFC041E4CD1079B5E491B8862
:10B260001A1D002D30D14A80059B5B4C5A89631909
:10B270001A716B1C9BB2E318120A1A71162306A8E6
:10B2800032881B1879890598FCF722FDFF21AA1C3A
:10B290002E1D03350B00059092B2B6B2ADB2002858
:10B2A00003D006ABDB8AD9B21B0AA218651911714B
:10B2B0002B714C4D301D2A884949201800F048FC5C
:10B2C0002B88F618B5B2A1E74988914207D17A8850
:10B2D00006995200525AEB18053A9A42C4DC3E4C89
:10B2E0002800618800F0BCFB207021007888FAF704
:10B2F0005FFED1E5002DF2D13E89BFE6162606ABF2
:10B30000F61831003889FCF76FFC3D000400FA356F
:10B3100000282DD0037A9B060CD400227B89398922
:10B32000788800923A000C32FFF7E8FB041E10D038
:10B330003E8915E03088FFF741FB00281AD083686A
:10B34000002B17D02100122278889847041EE4D0E1
:10B35000EEE72B78002B02D17888FAF739FE002629
:10B360002B78002B00D097E5002C00D194E585E6E2
:10B370000124DDE70E24DBE7162506ABED182900D6
:10B380003889FCF731FC041E47D0037A9B0611D4A0
:10B39000154A7B881188994203D01448814207D10D
:10B3A0001380134BF2261D780023D9B2A94221D372
:10B3B0000924A1E72888FFF701FB00282FD0836824
:10B3C000002B2CD02100122278889847041EDFD051
:10B3D00092E7C0465864FF1F2868FF1F2A68FF1FB6
:10B3E0001C69FF1F0C6AFF1F086BFF1FFFFF000097
:10B3F000066BFF1F31005943546801336018615ACE
:10B400000029D2D13C0008342100F22200F0A0FB38
:10B4100021007888FAF7E4FD3EE501246CE70E246C
:10B420006AE71D4B1A887B889A4231D07888FAF7F0
:10B43000E1FD31E5F223059851684343CD18C95A1F
:10B4400000291FD03B7A012B0BD16C88AB88788800
:10B45000AA1D0094FFF752FB041E02D000233B728A
:10B460002E88F2220021280000F0AAF900232B8068
:10B47000059B0133DBB20593084B05991B78064AFF
:10B480008B42D7D801235B421380002CCED0F5E548
:10B49000002634000596EFE7086BFF1F066BFF1FC1
:10B4A00070B504000E001500FFF796FA031E08D1D0
:10B4B00031000548FFF790FA03001120002B02D05D
:10B4C0001C8000209D7070BDFFFF0000F8B50B4F81
:10B4D00006003B780D001400FF2B0ED00A2000F070
:10B4E00037F9011E09D0B123038000234680037180
:10B4F000C5800481387800F01BF9F8BD2D44FF1F8A
:10B50000F7B50F0008A90600088809A90B240988C7
:10B51000002821D10234022B1ED1557813782D0238
:10B520001D432B008B4301937334002B14D1FB6814
:10B53000300019000093FFF74FFB019C85420BD0B0
:10B540002A0030000099FFF7ABFF041E04D12A0047
:10B5500030007989FFF7BAFF2000FEBDF0B50E7804
:10B5600085B003900AA805880120022E0DD14C68F1
:10B570002778647824023C43054FBC4205D10398E8
:10B58000DBB201960095FFF7BBFF05B0F0BDC046EA
:10B5900002290000034B10B51B68002B00D0984710
:10B5A000FEE7C046146BFF1F07B501A8FFF7F2FFC7
:10B5B000044A05480021121A00F05AF9F8F71AF95E
:10B5C000FEE7C046186BFF1F3044FF1F000000005D
:10B5D00001B40248844601BC604700BF8B520100A1
:10B5E00001B40248844601BC604700BF350E00002C
:10B5F00001B40248844601BC604700BFC51D00007D
:10B6000001B40248844601BC604700BF291C000009
:10B6100001B40248844601BC604700BF25260000F3
:10B6200001B40248844601BC604700BF1930FF1FC7
:10B6300001B40248844601BC604700BF055E0000BB
:10B6400001B40248844601BC604700BFEDA500007C
:10B6500001B40248844601BC604700BFE117000006
:10B6600001B40248844601BC604700BFC521000008
:10B6700001B40248844601BC604700BF810E00004F
:10B6800001B40248844601BC604700BF350E00008B
:10B6900001B40248844601BC604700BF2D3BFF1F38
:10B6A00001B40248844601BC604700BF792DFF1FEA
:10B6B00001B40248844601BC604700BFD91B0000AA
:10B6C00001B40248844601BC604700BF9DA9000048
:10B6D00001B40248844601BC604700BF6DBC000055
:10B6E00001B40248844601BC604700BF017F0000EE
:10B6F00001B40248844601BC604700BF5118FF1FD7
:10B7000001B40248844601BC604700BFADAE0000F2
:10B7100001B40248844601BC604700BFDD660100F9
:10B7200001B40248844601BC604700BFCD4C010013
:10B7300001B40248844601BC604700BF594F010074
:10B7400001B40248844601BC604700BF8552010035
:10B7500001B40248844601BC604700BF1D4D010092
:10B7600001B40248844601BC604700BF01240000C8
:10B7700001B40248844601BC604700BFB54C0100DB
:10B7800001B40248844601BC604700BF5522000056
:10B7900001B40248844601BC604700BFD91AFF1FAC
:10B7A00001B40248844601BC604700BF311B000061
:10B7B00001B40248844601BC604700BFC12FFF1F8F
:10B7C00001B40248844601BC604700BF154D01002A
:10B7D00001B40248844601BC604700BFA54F010088
:10B7E00001B40248844601BC604700BF1147010014
:10B7F00001B40248844601BC604700BF090E000046
:10B8000001B40248844601BC604700BF4D1F0000E0
:10B8100001B40248844601BC604700BF3D4B0100B3
:10B8200001B40248844601BC604700BFDD520100FC
:10B8300001B40248844601BC604700BF193BFF1FAA
:10B8400001B40248844601BC604700BF3938FF1F7D
:10B8500001B40248844601BC604700BF1D4B010093
:10B8600001B40248844601BC604700BF9135FF1F08
:10B8700001B40248844601BC604700BFB70E000017
:10B8800001B40248844601BC604700BF8D1200002D
:10B8900001B40248844601BC604700BF413BFF1F22
:10B8A00001B40248844601BC604700BFE54800007F
:10B8B00001B40248844601BC604700BF4550000007
:10B8C00001B40248844601BC604700BF456B0100DB
:10B8D00001B40248844601BC604700BF75A900005E
:10B8E00001B40248844601BC604700BF7D18FF1FB9
:10B8F00001B40248844601BC604700BF51250000E6
:10B9000001B40248844601BC604700BF014C0100FD
:10B9100001B40248844601BC604700BF35550000B1
:10B9200001B40248844601BC604700BFC52DFF1F1B
:10B9300001B40248844601BC604700BF4551010084
:10B9400001B40248844601BC604700BF0132FF1FBA
:10B9500001B40248844601BC604700BF2932FF1F82
:10B9600001B40248844601BC604700BFC56D0100B8
:10B9700001B40248844601BC604700BF7139FF1F13
:10B9800001B40248844601BC604700BFD9490100A8
:10B9900001B40248844601BC604700BF156B01003A
:10B9A00001B40248844601BC604700BF554901000C
:10B9B00001B40248844601BC604700BF2951010020
:10B9C00001B40248844601BC604700BFC9A9000019
:10B9D00001B40248844601BC604700BFB14E00007C
:10B9E00001B40248844601BC604700BF9136FF1F86
:10B9F00001B40248844601BC604700BF6130FF1FAC
:10BA000001B40248844601BC604700BFA94601005A
:10BA100001B40248844601BC604700BF51470100A1
:10BA200001B40248844601BC604700BF21460100C2
:10BA300001B40248844601BC604700BF851F000076
:10BA400001B40248844601BC604700BFC94A0100F6
:10BA500001B40248844601BC604700BF4D38FF1F57
:10BA600001B40248844601BC604700BF090E0000D3
:10BA700001B40248844601BC604700BFC9260000EB
:10BA800001B40248844601BC604700BFED39FF1F86
:10BA900001B40248844601BC604700BF7918000029
:10BAA00001B40248844601BC604700BF5D17000036
:10BAB00001B40248844601BC604700BF9D35FF1FAA
:10BAC00001B40248844601BC604700BFF54E010046
:10BAD00001B40248844601BC604700BFD92FFF1F54
:10BAE00001B40248844601BC604700BFF30E000069
:10BAF00001B40248844601BC604700BFF94C010014
:10BB000001B40248844601BC604700BF595201009D
:10BB100001B40248844601BC604700BF0539FF1FDD
:10BB200001B40248844601BC604700BFC135FF1F15
:10BB300001B40248844601BC604700BF691F000091
:10BB400001B40248844601BC604700BF193AFF1F98
:10BB500001B40248844601BC604700BFE94C0100C3
:10BB600001B40248844601BC604700BFED4A0100B1
:10BB700001B40248844601BC604700BF0D52010079
:10BB800001B40248844601BC604700BF4537FF1F2F
:10BB900001B40248844601BC604700BFC538FF1F9E
:10BBA00001B40248844601BC604700BF8538FF1FCE
:10BBB00001B40248844601BC604700BF2124000054
:10BBC00001B40248844601BC604700BFB352010083
:10BBD00001B40248844601BC604700BF434D0100E8
:10BBE00001B40248844601BC604700BF5933FF1FBF
:10BBF00001B40248844601BC604700BFE928000048
:10BC000001B40248844601BC604700BF6571010071
:10BC100001B40248844601BC604700BF091B000014
:10BC200001B40248844601BC604700BF056A0000B9
:10BC300001B40248844601BC604700BF3D180000C3
:10BC400000010103020203030403050206020702C6
:10BC5000080209030A030B030C020D000E030F0375
:10BC6000100311031303140315001600C53B001144
:10BC7000F93B0011000000000200000082BC00112E
:10BC8000192A0F180A000000F1590000FD240000D5
:10BC9000414601002580001139A000118D7400116A
:10BCA000297E0011115300112DAE0011794F0011A2
:10BCB000B93D0011E93E0011000000001616000019
:10BCC00002000000CCBC0011F4FFF3FFD2FC000026
:10BCD0002940001100000000000000005475796147
:10BCE0000042312E34003030313500676974687598
:10BCF000622E636F6D2F7076767800544830350071
:10BD00000200000014BD0011292A282A272A262A09
:10BD1000252A242A0A180000E2040000710200000B
:10BD200078EC0000744000001027000060F0000074
:10BD300006640000204E0000000000000500000026
:10BD40001F501D00023CB40000011500140000004B
:10BD5000A1020000303132333435363738394142B0
:10BD60004344454600000000155700116957001173
:10BD7000000000000200000080BD00116F2A6E2A42
:10BD80001A18EAD8BC80F0FC600000000000000037
:10BD90000000F303B59747D6F613F7D777E6F0A779
:10BDA000F474000001A00000000000006410B71D42
:10BDB000C8206E3BAC30D9269041DC76F4516B6BD9
:10BDC0005861B24D3C7105502083B8ED44930FF09B
:10BDD000E8A3D6D68CB361CBB0C2649BD4D2D38651
:10BDE00078E20AA01CF2BDBDFB349B5F800000809E
:10BDF00000100000000000008F6000111977001192
:10BE0000B3600011217B001137610011F77A001136
:10BE1000AD610011CD7A0011FF610011957C001118
:10BE200067620011957C0011996200114F7C00112E
:10BE3000AD610011857A0011256200112D7C001181
:10BE400000000000000000000B6300112D7C0011B9
:10BE50006D63001131770011052A042A012A002A96
:10BE600002290328012800280118001800000000FA
:10BE70000000000000000000000000870101020136
:10BE80000201010201020303040103010101010196
:10BE90000303020103000D000E0010001100130047
:10BEA0001401070108010A010B011C011D02040213
:10BEB00005020702080219021A021C021D030103EF
:10BEC000020317000201000504000807000B0A0026
:10BED0001716001D1C010201010504010E0D0111C0
:10BEE00010011413011716011A19020201020B0A9C
:10BEF000020E0D021110021413021716030504039B
:10BF00000807030B0A030E0D0001020307090A0BC1
:10BF10000E0F101112141718191A1B1F20212200BE
:10BF200075A7001131A800110000000002000000F8
:10BF30006ABE0011000000005DB5001100000000A5
:08BF40000200000068BE0011C0
:020000041FFFDC
:1000000000000000213D001188BC001184BC0011DB
:100010003C61FF1F00000000000000000000000025
:1000200000000000000000000000000000000000D0
:1000300000000000000000000000000000000000C0
:1000400000000000000000000000000000000000B0
:1000500000000000000000000000000000000000A0
:100060000000000000000000000000000000000090
:100070000000000000000000000000000000000080
:100080000000000000000000000000000000000070
:100090000000000000000000000000000000000060
:1000A0000000000000000000000000000000000050
:1000B0000000000000000000000000000000000040
:1000C0000000000000000000000000000000000030
:1000D0000000000000000000000000000000000020
:1000E0000000000000000000000000000000000010
:1000F0000000000000000000000000000000000000
:1001000000000000000000000000000000000000EF
:1001100000000000000000000000000000000000DF
:1001200000000000000000000000000000000000CF
:1001300000000000000000000000000000000000BF
:1001400000000000000000000000000000000000AF
:10015000000000000000000000000000000000009F
:10016000000000000000000000000000000000008F
:10017000000000000000000000000000000000007F
:10018000000000000000000000000000000000006F
:100190004D32FF1FAD30FF1FC1660100000000009F
:1001A000000000000000000000000000000000004F
:1001B000000000000000000000000000000000003F
:1001C000000000000000000000000000000000002F
:1001D000000000000000000000000000000000001F
:1001E000000000000000000000000000000000000F
:1001F00000000000000000000000000000000000FF
:1002000000000000000000000000000000000000EE
:1002100000000000000000000000000000000000DE
:1002200000000000000000000000000000000000CE
:1002300000000000000000000000000000000000BE
:1002400000000000000000000000000000000000AE
:10025000000000000000000000000000000000009E
:10026000000000000000000000000000000000008E
:10027000000000000000000000000000000000007E
:10028000000000000000000000000000000000006E
:10029000000000000000000000000000000000005E
:1002A000000000000000000000000000000000004E
:1002B000000000000000000000000000000000003E
:1002C000000000000000000000000000000000002E
:1002D000000000000000000000000000000000001E
:1002E000000000000000000000000000000000000E
:1002F00000000000000000000000000000000000FE
:1003000000000000000000000000000000000000ED
:1003100000000000000000000000000000000000DD
:1003200000000000000000000000000000000000CD
:1003300000000000000000000000000000000000BD
:1003400000000000000000000000000000000000AD
:10035000000000000000000000000000000000009D
:10036000000000000000000000000000000000008D
:10037000A9B500110000000000000000000000000E
:10038000000000000000000000000000000000006D
:10039000000000000000000000000000000000005D
:1003A000000000000000000000000000591AFF1FBC
:1003B000000000000000000000000000000000003D
:1003C000000000000000000000000000000000002D
:1003D000000000000000000000000000000000001D
:1003E000000000000000000000000000000000000D
:1003F00000000000000000000000000000000000FD
:08183800206FFF1F4118FF1F84
:10184000024981F3088802F057FB0000206FFF1F58
:1018500010B502F021FB072804D0122808D0022876
:1018600008D010BD044A0420136B01331363F8E75A
:101870000220F6E71420F4E70065FF1FF8B5070023
:101880000C0026002500503630785135002804D150
:101890000300287058342370F8BD2978CA00481E08
:1018A0008141A3183800A25C5B68C9B2FFF7D0FF82
:1018B00000280DD12B78DA00A218013350602B706C
:1018C0003378044A013B3370136A01331362D8E75B
:1018D0000123DFE70065FF1F5C234343074910B581
:1018E000C9180B0058331B78012B05D1FFF7C6FF31
:1018F000034A936A0133936210BDC0463465FF1FEB
:101900000065FF1F10B502F097FA064A0121130087
:1019100010CB4942D967044B136002F04DFB200005
:1019200010BDC04600E100E01000100010B504003A
:1019300002F082FA024B1C6002F03EFB10BDC04672
:1019400000E100E0431E5A425341A022F0B5D2010B
:101950005B421340154D164A40019B182A18127E0F
:101960008BB00191002A1BD01A000832D46F0022DC
:10197000E6B206AFE4B294420EDC2818C369002B2D
:1019800008D0019902AA117106AA049202AA16733C
:1019900003A898470BB0F0BD1978B9540132EAE7B3
:1019A0001A7D1A7806AB01261A70E6E7C067FF1F9A
:1019B00000400040F0B5254B04004001C25C85B0FA
:1019C000002A2BD01A18117E002927D0917E0029D9
:1019D00024D01179022921D11689D788D168F51B25
:1019E000ADB22A1C102D00D9102292B2BE4217D1DE
:1019F0001818012303710023C269C38003819A422E
:101A000006D06846032103730171029301A8904731
:101A10000820002C00D0192001F0FEFA05B0F0BD1E
:101A2000013C65426C41A0256442ED012C40084D0B
:101A30001B186419074D0633013A92B2AA42EDD041
:101A40001888461C1E80085C2070F5E7C067FF1FE1
:101A500000400040FFFF00000F220E4B10B59868B9
:101A6000104002380A280BD802F060F80D0A0B0A61
:101A70000A110A0A0A0A060002210020FFF762FF83
:101A800010BD0121F9E70020FFF794FFF8E7DB6FB5
:101A9000F6E7C046004000400F220E4B10B5986894
:101AA000104002380A280BD802F040F80E0A0B0A40
:101AB0000A120A0A0A0A060002210120FFF742FF61
:101AC00010BD01210800F9E70120FFF773FFF7E7D8
:101AD000DB6FF5E70090004013B5334C2378072BFC
:101AE0003DD8324B1A78324B002A39D180221968FE
:101AF00052020A431A60252001F0C4FE20232D4A19
:101B000011680B43802113606B460422C9050868E5
:101B10000733104228D080210422C905C86810422A
:101B20002ED080212020C905CA688243CA601422B1
:101B30001A701A78002A2FD18021C905C86820326E
:101B40000243CA6014221A701A78002A28D11A4B4C
:101B50001A7D22785A601D221A705932DA6013BD3C
:101B60001A6816490A40C5E7086802430A60142249
:101B70001A701A78002ACED01A78013AD2B2F7E752
:101B8000C8680243CA6014221A7019784A1ED2B279
:101B90001A700029F9D1C4E71A78013AD2B2C7E71E
:101BA0001A78013AD2B2CEE76843FF1F3044FF1FD4
:101BB0003CF000406043FF1F00200040FFFFFEFF9D
:101BC000564B70B51B68012B03D1554A936D0133F9
:101BD000936502F029F9534B534A1860534B544C08
:101BE0001A600123534A1360534A13602378002B71
:101BF00006D006225149524802F0DEF80023237035
:101C0000504A514B10681B78C1B2002B0ED14F4C7B
:101C1000C0B223785BB2002B4FDB237824785BB211
:101C200064B21B0424021B191B1813600B1C5029DF
:101C30004ED95023464A47491078DBB2FF2202288A
:101C40004BD10868444C454D267890432A789642FB
:101C500054D9227824782E78023B5D10A31B6B4365
:101C60005201D31A10335B111843086001F074FF5E
:101C7000031F012B45D83A4B1B78002B06D0394B5C
:101C80001B78002B02D0002002F046F8A122364B30
:101C900092009978354B4A431B689B188322920027
:101CA0009B181B78033B012B03D8AF20400002F0A8
:101CB00003F801222E4BDA8270BD237824785BB2C0
:101CC00064B2FF33FF341B0424021B190138ABE755
:101CD000CAB2022AAED20223ACE70868254C264DD0
:101CE000267890432A78964208D9227824782D784D
:101CF000023B5B10641B63435201B2E72378DBB203
:101D0000B2E70228D5D11D4B1B78013B022B03D92A
:101D10001B4B1B78022BCCD16C20C8E79809FF1F06
:101D2000FC0FFF1F3864FF1FFF3F0000141003402B
:101D30003C64FF1F0C10034000100340D50BFF1F35
:101D40007211FF1FB40003408C09FF1F680AFF1FB8
:101D5000490AFF1F94000340460AFF1F470AFF1F5E
:101D6000F908FF1F2209FF1F300DFF1F3409FF1F55
:101D7000BC0BFF1F440AFF1F450AFF1F1C09FF1F62
:101D80002309FF1F10B502F02FF80022014B1A8023
:101D900010BDC0463464FF1F10B501F02DFFA12116
:101DA000054A89009478054A61431268044B521829
:101DB000528C1A8010BDC046300DFF1F3409FF1F22
:101DC0003464FF1F10B50D4B0D4A9978A1239B0079
:101DD0004B431268D218531DD97F0A4B1B88994276
:101DE00009D2441C07D0C82805D0D2695B1A5A43CF
:101DF000054B5343C01801F0EFFE10BD300DFF1F1F
:101E00003409FF1F3464FF1F7102000070B5244DB8
:101E10002B68002B28D002F087F82B68D8402B685D
:101E20000400002B27D002F0AFF82B68D8401D4BE0
:101E30001D4A9978A1239B004B431268D118D25CAC
:101E400091239B00002A20D0CA580132CA50174B58
:101E500017491B680868834214D3D23B181A012A19
:101E60001AD0144B186070BD02F05EF8124B19685E
:101E700002F062F8D3E702F087F80F4B196802F01E
:101E80005BF8D4E70D495B18E8E7CA500C4B1B68B8
:101E9000DB68E418201AE4E7F530FF30E1E7C046DC
:101EA0001C08FF1F300DFF1F3409FF1F9C09FF1F77
:101EB0003864FF1FA009FF1F1808FF1F2DFF3F00F8
:101EC0004064FF1F70B504000D00282916D10300DF
:101ED000A433C2881B889B1A0B4A9BB293420DD92C
:101EE00006006A3605223100653001F07DFE0028CB
:101EF00004D13100200002F057F870BD2900200005
:101F000001F0F2FEF9E7C046FE7F0000F8B50500DB
:101F1000012002F019F8134CA36AA26A9342FBD184
:101F2000114E336001F028FE10490300086010488C
:101F3000426894460F4A17680022BC4501D24268A5
:101F4000BA1A0D4802603268AD18A422E562606AD0
:101F5000520302436262094A1278002A01D00F3B01
:101F60000B60F8BD00F00040340AFF1FE408FF1FBB
:101F700028100040180AFF1F1C0AFF1F1C09FF1F22
:101F800070B580241025E405A3682B43A36001F0FD
:101F9000BBFFA368AB43A36070BD0000F7B516009C
:101FA00080221C001023D2050191916805000B438B
:101FB000936000225A4BD7301A6001F0BDFE9D237A
:101FC0002A002F009B00EB58CA3201210092FC37F7
:101FD000002B01D00021009A386801F035FF29005C
:101FE000009BCB311A784F4BD3351A604B780A7867
:101FF0001B0213438A7812041A43CB781B0613433F
:10200000494A1BBA13604B790A791B0213438A7938
:1020100012041A43CB7931001B061343434A1BBAFF
:1020200013606B782A781B021343AA7812041A43B0
:10203000EB781B0613433E4A1BBA1360019A330226
:1020400013433C4A13603C4B22001B1B9C46032954
:102050003DDCB3089A0013005142B21A032A46D15C
:10206000354AE018511A827840781204000202437F
:10207000E05C043302430A600022FF2B4BDDF022B8
:102080002E4B12011A600F222D4B1A602D4A136835
:10209000002BFCD00023224A27491360091B321D64
:1020A0000B191B68043A180A23706070180C1B0E79
:1020B000A070E3700434002AF2DC802210213B6817
:1020C000D20501333B6093688B439360F7BD634651
:1020D000D578981893782D061B042B43157804396E
:1020E0002B43557804322D022B430360AFE7022ABD
:1020F0000AD1114AE05C511AE218527812020243E6
:102100000A6004339BB2B7E7012AB5D10A4A521AD2
:10211000E15C1160F5E7084959180A600433ACE73F
:10212000000004403C0004403800044034000440F7
:10213000300004400C00044000010440040004404E
:102140001000044014000440F7B5150080221C0064
:102150001023D2050091916807000B439360002380
:10216000654AD730136001F0E7FD9D233E009B00D8
:10217000F9583B00CA363200FC33002900D07FE01A
:10218000586801F061FE390032785C4BCB311A603F
:102190004B780A781B0213438A78AC4612041A4320
:1021A000CB78281D1B061343554A1BBA13604B7985
:1021B0000A791B0213438A7912041A43CB791B064E
:1021C0001343504A1BBA13604B7A0A7A1B0213431B
:1021D0008A7A12041A43CB7A21001B0613434A4A17
:1021E0001BBA1360009A2B021343484A1360220063
:1021F000474B1B1B0093009BCE785B1801938B7899
:1022000036061B0433430E78043833434E780431CA
:1022100036023343019E33600328ECDC0321A80817
:10222000431C9B002940800003292BD13849E51825
:102230005E18A9786D78E35C09042D0229431943DF
:102240003160030008330021FF2B2DDD314B324973
:1022500019600F21314B1960012327490B60304B66
:1022600019680029FCD006211B680B40042B20D0E4
:1022700080220020D20593680A318B439360FEBD13
:1022800001217DE7022908D121495D18E11849782B
:10229000E35C090219432960D3E70129D3D11C4922
:1022A0005918E35C0B60CCE7194818180160043337
:1022B000CAE7002310490B606346002B0CDC3B008F
:1022C000FC335A68102101325A608022D20593688B
:1022D00001208B439360D2E7009B9B181B68190A6F
:1022E00013705170190C1B0ED37004235B42917054
:1022F0009C440432E0E7C046000004403C00044037
:102300003800044034000440300004400C00044015
:102310000001044004000440080F000010000440C5
:102320001400044070B5061E19D002225A4B9B7946
:102330009343012B13D1594B1A78FF2A0FD15A78A6
:10234000FF2A0CD19A78FF2A09D1DA78FF2A06D120
:102350001A79FF2A03D15B79FF2B00D199E0504B0A
:102360000C201A78012A08D000224E4D1A702978C4
:102370000B00093B042B01D8212070BD4B1F012B02
:10238000FAD9454CA37B042B00D982E0A279032A19
:1023900000D97EE09A1ED2B2012A02D860881F2896
:1023A00077D9002E56D0012E73D1A0880128E3D012
:1023B000002907D1581E032803D801F0B7FB1217D4
:1023C00015122E702978481E032811D80025364B87
:1023D0001D602823237501F057FDA84227D0A58052
:1023E000CAE702212970EDE70421FBE70321F9E7A1
:1023F00007390129C0D82D490968C96A8906BBD5A2
:102400002B4908780028B7D1012A01D9002BB3D174
:1024100002230B708021274D2633890128782375EC
:1024200001F02AFC80212878890101F065FC012354
:10243000A380214B1B78002B0AD0FA2280211F4B4E
:1024400092001B8809025A431A4B187801F044FD88
:10245000002092E701F0F0FC2B78A680073B012BCF
:1024600003D917482E7001F087FC114B114C1A78D4
:10247000002A06D080210022207889011A7001F0FC
:10248000FBFB01F099FD80212078090201F0F4FBAB
:10249000DEE7122071E7C046A60BFF1F6B09FF1F86
:1024A0001A09FF1F1C09FF1F4809FF1F4064FF1F77
:1024B0002309FF1F1B09FF1F2109FF1F2C09FF1FF5
:1024C0000010004010B5002901D001F08DFD10BDB5
:1024D000F7B5604B01919978A1239B004B435E4A6D
:1024E000060014681022E418D6235B00E058362357
:1024F000FF33E35C00279343222B41D1574B0F3A24
:102500001A600760012501F067FD019B1880E82330
:102510005B00E35C002B01D0B34258DD0023504F39
:10252000FB70AD33FF33E3581A68002A03D09B8851
:10253000DB439B071DD03823FF33E35C002B18D00F
:102540009B235B00E35C002B13D1D133FF33E35CAF
:10255000B3420EDAA4235B00E15AE018090A023103
:1025600001F0AAFC23000122FE33013E01351A8747
:10257000FA70E8235B00E35C002B2AD0A8B2FEBD12
:1025800003683D00002BBED081880430090A023167
:1025900001F092FCD6235B00E3581F60B2E72300F2
:1025A000B133BA00FF339858013781880430090AE3
:1025B000023101F081FCE8235B00E35CBB42EEDC0E
:1025C000E822F61AED1800235200A354A6E70027CC
:1025D000F1E7200001F038FB00281FD0002E1DDDA0
:1025E0007319882647190193B600200001F01CFDDD
:1025F0005A30800020184068013581880430090A6B
:10260000023101F059FC200001F0C6FAA359013350
:10261000A351BD4202D0019B9D42E6D1114BE35C28
:10262000002BABD095239B00E35C002BA6D00E4B78
:10263000E15A0029A2D00D4AA35C994202D9013384
:10264000A3549BE700231A212000A35401F0B4FAFD
:1026500094E7C046300DFF1F3409FF1F00140340EC
:10266000E010FF1F5A020000720200005E0200002C
:102670000D4970B54A6E0D4CD2038B69D20BA24244
:1026800006D80B4D0224AA4204D901F07DFB70BD8F
:1026900002246442E21815007E2425402242F4D030
:1026A000A3432B438B61F0E700F000400A200000B9
:1026B000FC1C0000F8B51D4B1D4F1A78002A10D1E4
:1026C000BA7B002A02D101321A7003E0032AFAD041
:1026D000022AF8D001F0D8FB00220120154B1A7015
:1026E000F8BD154B154D1C68154B9E7801232B70BA
:1026F0002878C0B200F0A2FBBB7B002B0BD101F00D
:1027000053FAA1239B007343E41883239B00E4182E
:1027100023782B70E4E7032B02D101F055FBF0E79F
:102720000020022BDCD101F09FFBEAE71C09FF1F10
:10273000A60BFF1F2309FF1F3409FF1F490AFF1FB4
:10274000300DFF1FF0B587B00EAD2F780FAD2D788F
:102750000593AC46634614000E4D0CAA12782E78F1
:1027600003930D9B009201932200059B029701F0B9
:102770006BFC2E70012C01D0042C08D1802206495C
:102780008B889343054A1278D20113438B8007B09C
:10279000F0BDC0461C09FF1F6C11FF1F7809FF1F09
:1027A0000B001B3B70B504003020E02B0DD813004C
:1027B000E025493BFF3B9BB2ED00AB4205D8034B04
:1027C000200019825A8201F01FFA70BD8410FF1F89
:1027D00010B501F029FB054B00205B68052B04D9DF
:1027E000034A5268D20200D4980810BD001000407D
:1027F000FCE100E070B501F01FFB0D4B1B68FC33E2
:10280000DC691D6AFFF7E4FF6419844204D2094BB6
:1028100001241B68002B07D004220024064B1A70E9
:10282000064A93690133936101F0C6FB200070BD35
:102830004064FF1F9809FF1F2309FF1FFC0FFF1FA4
:1028400070B50C4D2B68FC335C6A01F0F5FAFFF7AC
:10285000BFFF2B680025FC339B6AE318834204D238
:10286000054B1B68AB4200D1051B01F0A5FB2800FE
:1028700070BDC0464064FF1F9809FF1FD722044B5C
:1028800092009B5810B5002B00D0984710BDC04651
:102890000000FF1F10B501F0D3F8FFF7EFFF274945
:1028A000274BCA6D274C1A4084235B001343CB652A
:1028B000254B1B68186A01F047FB244B244A1A6019
:1028C000244B254A1A60A022244B52001A60244B44
:1028D000187801F051FB2000224901F0F5F900239E
:1028E000A3600233A360204B2049236003232048C8
:1028F000A36001F0E9F910221E4BFF201A6080222C
:1029000052031A60802292031A60802212041A6015
:1029100001F002FA012001F017FAFA20400001F05C
:10292000A3F9582001F0C8F9134801F07DF90120FE
:1029300001F012FA072001F04FFA10BD00F000403C
:1029400000FEFEFF141000404064FF1F0000034023
:102950000180063DBC00034034080000A400034091
:102960004A0AFF1F71020000C3090000FFFF3F0079
:102970002810004000E100E030750000674E336829
:1029800088331B6883F3088801F00EFA644A6549AE
:10299000136800200B401360634B644A1B6893422A
:1029A00000D1A6E001F030FB0221614A13688B439D
:1029B0001360FFF76FFF5F4B5F4C1878C0B201F0F8
:1029C0004BF90023A3600233A3605C4B012023601A
:1029D00001F0BAFA0323A36001F066F9040001F0E4
:1029E00023FA050001F060F9554B186001F094FAE4
:1029F000544B1968621A531EA14200D21300802260
:102A0000D203934201D39B029B0A3268D16AC90761
:102A100000D471E04C491C0C09689BB24C435943EB
:102A20002402090A641803264849FC3293680A689C
:102A300047489B1A474A0768126847499B18474A04
:102A40009A1833409208DB190A600360042B03D9FB
:102A5000013233400A6003600E684149A619300014
:102A600001F06AFA3F4F3E493B68C3183B603000B3
:102A7000019301F0F1F93C4E306808183849306094
:102A8000884205D9019B01333B6001F0E5F93160D3
:102A900001F062FA354B1B78002B0DD001F0C4F920
:102AA000334B621B196812188A4232D24919091B2A
:102AB000091A304801F008F92F4E337A002B0ED056
:102AC00001F0B2F9621BF1681218914224D9491938
:102AD000091B091A294801F0F7F800233372284B23
:102AE00083F3088801F050F8002001F08DFA01F01E
:102AF0000BF901F089FA5CE7DC0199000234641AF1
:102B00005900641A09214B438033CB40A408E418D0
:102B100089E7FA218900CCE71A49DBE74064FF1F07
:102B20001CF00040FFFFC1FF0C0AFF1FB64121034C
:102B300010000040490AFF1F14100040C3090000A4
:102B4000100AFF1F340AFF1F380AFF1F200AFF1F49
:102B5000280AFF1F1C0AFF1F240AFF1FC4090000C8
:102B6000710200006008FF1F2C0AFF1F1C09FF1FD5
:102B7000E408FF1F00100040740BFF1F3C100040D2
:102B800000000020DC050000A022054B92009B58AD
:102B900010B5002B01D0984710BD01F015F8FBE7E8
:102BA0000000FF1FA122054B92009B5810B5002B7F
:102BB00001D0984710BD01F007F8FBE70000FF1FA8
:102BC000A222054B92009B5810B5002B01D09847CC
:102BD00010BD00F0F9FFFBE70000FF1FA322054B2B
:102BE00092009B5810B5002B01D0984710BD00F003
:102BF000EBFFFBE70000FF1FA422054B92009B5850
:102C000010B5002B01D0984710BD00F0DDFFFBE7A9
:102C10000000FF1F70B501F007F94F4B186001F07D
:102C2000D3F90400C30702D401F0B6F870BD002246
:102C30004A4B1A604A4B18780138042829D800F00A
:102C400075FF0320181C2400200001F0D5F901288D
:102C5000ECD0444C2378042B6ED101F09DF9002870
:102C6000E4D000F0D9FF582001F026F802232370A9
:102C7000DCE7200001F038F9E9E7200001F054F822
:102C8000E5E7200001F070F8E1E7200001F0D4F959
:102C9000DDE700F061FF0500012808D1324B1B7809
:102CA000053B012B03D82000FFF76EFFD1E72D4B2A
:102CB0001B78022B01D0052B20D1022D28D12B4BC4
:102CC0009B7BAB431CD12000FFF76CFF264B187891
:102CD0000128BED16405BCD4244925224B7B034284
:102CE00005D1233A13405A42534126331A000B7D33
:102CF0009342AED9322001F08FF8AAE7022D07D116
:102D0000194B1B78052B11D12000FFF759FFDDE788
:102D1000012D0BD1012B03D12000FFF75FFF98E7B6
:102D2000062B03D12000FFF767FF92E7200000F099
:102D30004BFF022D8DD1C9E7032B04D10C4B987C9E
:102D400001F09AF872E7072B00D06FE7094B987BE8
:102D500000F072FF6AE7C0469C09FF1F9809FF1F39
:102D60009009FF1F2309FF1F1C09FF1FA60BFF1F50
:102D7000BC0BFF1FD40BFF1FFA210A4B0A4A490064
:102D80001A640A4A5A500A4A04395A50094A083100
:102D90009A64094A5A50094A5C315A50084ADA661C
:102DA0007047C0460000FF1F4527FF1F4128FF1F37
:102DB000F527FF1F2523FF1FB526FF1FC51DFF1F7A
:102DC000991DFF1F10B500F099FE10BDF7B50B0C53
:102DD000FF270122009300233C001E001D009446A3
:102DE000019089B262469A40100008401841361896
:102DF000B6B2FF2F02D1012E00D19FB2009802403F
:102E00001A41AD18ADB2FF2C02D1012D00D19CB2F8
:102E10000133102BE6D10320012E07D1012D04D15F
:102E2000019B2401E4191C700138FEBD102EFCD159
:102E30000238102DF9D00230F7E700008023F7B5F3
:102E40009C46264B264F01932649274A274D284C5E
:102E5000284B02281AD1604638600868264E304058
:102E6000802636033043086001990978002909D18A
:102E70001660224A2A60224A2260E02219689143A1
:102E8000A03A1BE08021C9021160F2E766463E606D
:102E90000F68194E3E408027FF023E430E600199A5
:102EA000097800290DD1176001280ED1154A2A6032
:102EB000154A2260E02219689143C03A0A431A6019
:102EC000F7BD802189021160EEE7E0210F4A02433D
:102ED0002A600F4A22601A688A43F0E74B0AFF1FF4
:102EE000E0000340D800034090000340000003408E
:102EF0005000034040000340FFFFE3FF0280063D17
:102F0000804508220180063D8066082200800698E0
:102F100080550822F8B51E4B80261A680020140040
:102F20003440324232D11A681A4F32431A600122B9
:102F30003B68063093433B6001F006F80122164DD2
:102F40002B681E432E603B680A2613433B60802794
:102F5000BF00124B1B683B4211D1013EF6B2FF2E5F
:102F600009D17E220E4B1C682B68E40B144093435E
:102F700023432B6005E0082000F0E6FFE9E7002E80
:102F8000EFD180222B68600893432B60F8BDC046C8
:102F9000C4F000405CF0004018F0004068F00040D1
:102FA00060F0004010B500F027FF01215820034ACF
:102FB00001F032F8FFF7AEFF10BDC046600AFF1FF8
:102FC00010B578220021034800F01EFF00F07CFFBE
:102FD000002010BD4867FF1F70B5040000F02CFFF3
:102FE00000230C200B4A010059438D18515C002925
:102FF0000DD0A14208D1012300246B7000F0B4FF72
:1030000000F0DAFF200070BD01330A2BEBD112244F
:10301000F6E7C0464867FF1F70B5040000F00CFFDC
:10302000002319001D000D4A1078002806D0A04288
:103030000CD1557001310C320A29F5D1002B0AD17F
:1030400000F042FF00F0B8FF002070BD5078461E2F
:10305000B0411B18EEE700F087FFF3E74867FF1F5A
:10306000F7B504000C20002384460E4D01926746FC
:103070005F43E85D7E19A04212D000280BD10A4BB5
:103080009C4662461B7808331370019B70707C5518
:103090007160B360FEBD01330A2BE8D10320F9E76C
:1030A0000720F7E74867FF1F4467FF1F8020F8B538
:1030B000484BC0051B68C1248360474BFF251A6835
:1030C000012313434361454BA4001A68444B40213C
:1030D0001A60444B1A68444B1A60444B1A59AA436D
:1030E0001A51C52292009E58AE4331438026995012
:1030F0009F583F49F6010F403E439E509E588027FF
:103100003602360A3043985080201A5900020A408D
:1031100002431A5104341A59364E3F043240802675
:103120003A431A511A5936061202120A32431A51F8
:1031300008341A5980260A4002431A51C3229200C9
:103140009F58B446AF4337439F509F58294E0F4076
:1031500007439F509F5837408026360437438026C8
:103160009F509F5836063F023F0A37439F50C02268
:103170001F59AF433A431A511A591202120A164301
:10318000C6221E5192009C58AC4365462C439C506D
:103190009C5800250C4020439850C72080001A58A6
:1031A000154C1140C02212020A431A50134B1B78CF
:1031B000DB08AB4201DC0020F8BD2378002B06D0F1
:1031C000A368002B00D0984701350C34EEE712209D
:1031D000F2E7C0466443FF1F6043FF1FB0F00040AA
:1031E0004067FF1FB4F000403C67FF1F00E100E0B4
:1031F000FF00FFFFFFFF00FF4867FF1F4467FF1F3F
:10320000030010B51F2809D8072200201340072407
:1032100004490A78A24313430B7010BD0023062013
:10322000F5E7C0464467FF1F054B06491B780A684F
:1032300005485B0702401B0B134300200B607047DF
:103240004467FF1F1CF00040FFFFC1FF70B50C2555
:10325000FFF7EAFF0A4B1C780A4BE4086543ED18B8
:10326000002C01D1200070BD2B78002B06D06B689C
:10327000002B00D09847013C0C3DF1E71220F2E70B
:103280004467FF1F3C67FF1F1FB5002102220B0090
:1032900001910091052000F007FE02230B490A6806
:1032A0001A42FCD120230393039B5A1E0392002B46
:1032B000FAD1074A1368002BFCDA0B246C44200077
:1032C000012100F0C9FE207804B010BD90C8004074
:1032D00000C8004013B504000A4B0193019B002B6A
:1032E00001D1112016BDFFF7CFFF23000340044298
:1032F00005D0052000F028FE019B013BEDE71800FA
:10330000F0E7C046FFFFFF0707B500F095FD8022FC
:103310000821D205936A0191002B01D107399162EE
:1033200002210C4A11600199481E01900029FAD12E
:1033300003311160053101910199481E0190002966
:10334000FAD11160002B02D18022D205936200F0E5
:1033500033FE07BD00C00040F0B52D4C89B0237886
:10336000002B4FD1FEF7CEFA02232A4F03903A6882
:103370001A42FCD120230693069B5A1E0692002B6C
:10338000FAD1254E3368002BFCDA0120FFF7A2FFAB
:10339000011E02D0112009B0F0BD030003220190EC
:1033A000009005AD9F2000F07FFD0321280000F074
:1033B00053FE02233A681A42FCD120230793079B4D
:1033C0005A1E0792002BFAD13368002BFCDA012039
:1033D000FFF780FF0028DDD10398FEF7A7FAAA784F
:1033E0006B7811041B020B4329780B4363601300B5
:1033F000113B0A49052B07D801239340A3600B60BA
:10340000012323700020C6E780231B03F6E7C04694
:103410004C43FF1F90C8004000C800409808FF1FA1
:103420001E4B30B55A6818781D4B85B0D3185942D9
:103430004B4101210093002300F096FB194B1A4ADF
:1034400002259A6300221A6510325A658022C4212F
:103450009D65164B1648D202DA6789004258154B13
:1034600080241A4080231B041343435064234120CB
:103470000393E40500F006FA402000F003FA6562C9
:10348000039D6B1E0393002DFAD103236362FFF7A4
:103490003BFFA562FFF760FF05B030BD5843FF1F3B
:1034A00095FFFEF700C80040050001FF04E100E0C1
:1034B00000E100E0FFFF00FFF0B585B00700FEF778
:1034C00021FA022305002D4C22681A42FCD1202348
:1034D0000093009B5A1E0092002BFAD1284E3368AD
:1034E000002BFCDA0120FFF7F5FE002803D01124A1
:1034F000200005B0F0BD234B2360022322681A424E
:10350000FCD120230193019B5A1E0192002BFAD17A
:103510003368002BFCDA0120FFF7DCFE0028E6D13F
:10352000194B1F60022322681A42FCD12023029308
:10353000029B5A1E0292002BFAD13368002BFCDA50
:103540000120FFF7C7FE0028D1D1104B23600223D2
:1035500022681A42FCD120230393039B5A1E039234
:10356000002BFAD13368002BFCDA0120FFF7B2FE02
:10357000041EBCD12800FEF7D9F9B9E790C8004075
:1035800000C8004001000006A8C8004001800001FA
:1035900010B50020FFF790FF10BD000010B5064BDE
:1035A00018705960FFF73CFF00211320034AFFF712
:1035B00057FD002010BDC0465843FF1F2134FF1F98
:1035C000F0B5040085B003920291FEF79BF98822C2
:1035D00063035B0B52051A438023DB059D6A80233E
:1035E000274F0092BA68002601901B039A420CD91B
:1035F000F82326001B041E401C4206D08022214BCB
:1036000052025E6219680A431A60002D0BD100F065
:1036100013FC02221C4B1A608023DB055A62013A1C
:103620009A6200F0C9FC0023039A934220D1002D36
:103630000AD100F001FC144B03221D608023DB053E
:103640005A629D6200F0B8FC8023BA681B039A425C
:1036500008D9002E06D000220A4B0C495A621A687B
:103660000A401A600198FEF761F9002005B0F0BD2C
:10367000009A0299D2181278CA540133D4E7C0468E
:103680004C43FF1F00C8004000C00040FFFFFEFF8A
:10369000F0B587B0029103920400FEF733F9019070
:1036A00000F0CAFB802302250122234EDB05356092
:1036B0005D629A6200F080FC204F3B682B42FCD197
:1036C00020230493049B5A1E0492002BFAD11C4D14
:1036D0002B68002BFCDA0120FFF7FCFD002802D04C
:1036E000112007B0F0BD2000039A029900F0CCFA37
:1036F000022304003A681A42FCD120230593059B5B
:103700005A1E0592002BFAD12B68002BFCDA0120FF
:10371000FFF7E0FD051EE3D100F08EFB80230322BE
:10372000DB0535605A629D6200F046FC0198FEF7A9
:10373000FDF8E0B2D5E7C04600C0004090C80040A8
:1037400000C80040F0B5802489B00600FEF7DAF822
:10375000E405A36A02250393029000F06DFB0123A8
:10376000304F3D606562A36200F026FC2E4C23685A
:103770002B42FCD120230593059B5A1E0592002B5A
:10378000FAD12A4D2B68002BFCDA0120FFF7A2FDAD
:10379000002803D01124200009B0F0BD244B236081
:1037A000022322681A42FCD120230693069B5A1E4C
:1037B0000692002BFAD12B68002BFCDA0120FFF7D0
:1037C00089FD021EE6D11B4B03211E600300019000
:1037D0000090202000F068FB022322681A42FCD1EE
:1037E00020230793079B5A1E0792002BFAD12B68C0
:1037F000002BFCDA0320FFF76DFD041ECAD100F098
:103800001BFB80230322DB053C605A629C6200F0B4
:10381000D3FB039B002B01D1FFF776FD0298FEF747
:1038200085F8B8E700C0004090C8004000C80040DC
:103830000100000694C8004007B50002019104226F
:10384000000A01A9FFF724FF0EBD000073B50500B3
:1038500005240B4AA3005B429B1819686B46DE1DCA
:103860003000FFF7B3FA022804D133782B55013C1E
:10387000EFD276BD052CFCD00128FAD10230F8E752
:10388000140900111F2807D8012380228340D20584
:1038900091680B43936070473F2808D8012380222A
:1038A00020388340D20551690B435361F3E75F2809
:1038B000F1D80123802240388340D205116A0B439E
:1038C0001362E8E71F2807D8012280218240C9053A
:1038D0008B6893438B6070473F2808D80122802172
:1038E00020388240C9054B6993434B61F3E75F2859
:1038F000F1D80122802140388240C9050B6A9343E8
:103900000B62E8E71F2810D880230200DB05153A78
:103910001968012A06D820229143196019680A43C0
:103920001A60704701228240F6E73F2811D88023B1
:103930000200DB05353AD968032A06D810229143E4
:10394000D960D9680A43DA60EBE701222038824067
:10395000F5E75F28E5D842238022181A413B8340CF
:10396000D205516A99435162516A0B435362D8E7B9
:1039700010B50400012813D1A022184992050B6844
:103980005B015B0913430B60154B164A1968114024
:10399000154A0A431A60402219680A431A6010BD8A
:1039A0000028FCD101000A2000F076F921000B204C
:1039B00000F072F9C0220A4B920019680A434021B4
:1039C0001A601A688A431A60B022044912060B680A
:1039D0005B015B0913430B60E1E7C04614F0004054
:1039E0001CF000407F00FEFF80FD010072B6074A18
:1039F0001368013313600422054B1A600023054A43
:103A000013608022D2055360FEE7C0467808FF1F8E
:103A1000C0F00040C4F0004005490B68002B05D100
:103A2000044A0A6004490A60044A13607047C046A9
:103A3000140AFF1F841E0000380AFF1FC4F0004054
:103A40000023034A1360034A1360034A136070475C
:103A500054F0004040F1004044F10040002310B514
:103A6000184C8AB0009301932378012B27D0694624
:103A7000012000F031F9002817D1009B1249029370
:103A8000019B06AA0393114B02A81B680493104BD9
:103A90001B68059300F038FA10220E4906A800F0C2
:103AA000A3F8002804D1FF23237000200AB010BD22
:103AB0000123094A074902A8237000F025FA0120D2
:103AC000F4E7C0464464FF1F1029001108290011C3
:103AD0000C290011202900114864FF1F13B501248F
:103AE0006946012000F0F8F8034B00940193FFF7BA
:103AF000B5FF200016BDC046BB0B000010B5FFF798
:103B00009FFFFFF7EBFF002802D0024B984710BD44
:103B1000FEE7C046E1A2000002B471464908490030
:103B2000095649008E4402BC7047C04602B4714633
:103B300049084900095C49008E4402BC7047C046F0
:103B400003B47146490840004900095A49008E44AF
:103B500003BC70470000000001B40248844601BC69
:103B6000604700BFDD0C010001B40248844601BC7F
:103B7000604700BFC56D010001B40248844601BC26
:103B8000604700BFBD5C010001B40248844601BC2F
:103B9000604700BF7997000001B40248844601BC29
:103BA000604700BF5976010001B40248844601BC59
:103BB000604700BFE9F6000001B40248844601BC3A
:103BC000604700BF53B9000001B40248844601BCFD
:103BD000604700BFE917010001B40248844601BCF8
:103BE000604700BF8937010001B40248844601BC28
:103BF000604700BFCD4C010001B40248844601BCBF
:103C0000604700BFF9ED000001B40248844601BCE2
:103C1000604700BF116E000001B40248844601BC39
:103C2000604700BF6DF6000001B40248844601BC45
:103C3000604700BF8D11010001B40248844601BCF9
:103C4000604700BFC1F7000001B40248844601BCD0
:103C5000604700BF71B0000001B40248844601BC57
:103C6000604700BF8914010001B40248844601BCCA
:103C7000604700BF8512010001B40248844601BCC0
:103C8000604700BFB352010001B40248844601BC42
:103C9000604700BF9573010001B40248844601BC2F
:103CA000604700BF09A2001101B40248844601BC6C
:103CB000604700BF156B010001B40248844601BC97
:103CC000604700BF7912010001B40248844601BC7C
:103CD000604700BF2D6C010001B40248844601BC5E
:103CE000604700BFE1AC000001B40248844601BC5B
:103CF000604700BF51B8000001B40248844601BCCF
:103D0000604700BF0D52010001B40248844601BC67
:103D1000604700BF8552010001B40248844601BCDF
:103D2000604700BFED6B010001B40248844601BC4E
:103D3000604700BF0534010001B40248844601BC5D
:103D4000604700BF8944000001B40248844601BCBA
:103D5000604700BF6911010001B40248844601BCFC
:103D6000604700BFE512010001B40248844601BC6F
:103D7000604700BFF535010001B40248844601BC2C
:103D8000604700BFC1A5000001B40248844601BCE1
:103D9000604700BFD1AE000001B40248844601BCB8
:103DA000604700BFDD0A010001B40248844601BC3F
:103DB000604700BFC9A9000001B40248844601BCA5
:103DC000604700BFE94C010001B40248844601BCD1
:103DD000604700BF75F8000001B40248844601BC8A
:103DE000604700BFF90D010001B40248844601BCE0
:103DF000604700BF8D82000001B40248844601BCC8
:103E0000604700BFED68010001B40248844601BC70
:103E1000604700BFB70E000001B40248844601BCF1
:103E2000604700BF6137010001B40248844601BC0D
:103E3000604700BFC95C010001B40248844601BC70
:103E4000604700BF75A9000001B40248844601BC68
:103E5000604700BF2144000001B40248844601BC11
:103E6000604700BF090E000001B40248844601BC4F
:103E7000604700BF19FA000001B40248844601BC43
:103E8000604700BF4DF9000001B40248844601BC00
:103E9000604700BFA9D8000001B40248844601BCB5
:103EA000604700BFE927000001B40248844601BC16
:103EB000604700BF496D010001B40248844601BC5F
:103EC000604700BFC115010001B40248844601BC2F
:103ED000604700BFADAE000001B40248844601BC9B
:103EE000604700BF8B52010001B40248844601BC08
:103EF000604700BF0934010001B40248844601BC98
:103F0000604700BFB1B5001101B40248844601BC4E
:103F1000604700BFDD3F000001B40248844601BC99
:103F2000604700BFC166010001B40248844601BC7D
:103F3000604700BFE90B010001B40248844601BCA0
:103F4000604700BF090E000001B40248844601BC6E
:103F5000604700BF0189000001B40248844601BCEB
:103F6000604700BFD544010001B40248844601BC4B
:103F7000604700BF21A9000001B40248844601BC8B
:103F8000604700BFEDA5000001B40248844601BCB3
:103F9000604700BF6D0B010001B40248844601BCBC
:103FA000604700BF01D7000001B40248844601BC4D
:103FB000604700BF85C1000001B40248844601BCCF
:103FC000604700BF9DA9000001B40248844601BCBF
:103FD000604700BFBD0B010001B40248844601BC2C
:103FE000604700BFCD0C010001B40248844601BC0B
:103FF000604700BFE9D4000001B40248844601BC18
:10400000604700BF0134010001B40248844601BC8E
:10401000604700BF016C010001B40248844601BC46
:10402000604700BF0167010001B40248844601BC3B
:10403000604700BFD9B0000001B40248844601BC0B
:10404000604700BFF935010001B40248844601BC55
:10405000604700BF9D6A000001B40248844601BC6D
:08406000604700BF3D71010043
:104068000200000066BE00110100000078BC0011CB
:104078000200000062BE001101000000A840FF1FFE
:104088000200000080BC001101000000BC61FF1F9D
:104098000200000060BE0011030000003061FF1F35
:1040A800120000000200000066BE001101000000BE
:1040B800C0BC00110200000062BE00110100000037
:1040C800BDBC001102000000CABC001103000000C2
:1040D8006B61FF1F0200000060BE001103000000BA
:1040E8008061FF1F0200000062BE00110100000095
:1040F800BCBC001102000000C8BC00110300000095
:104108004161FF1F0200000060BE001103000000B3
:104118006261FF1F0200000066BE0011010000007E
:1041280000BD00110200000062BE00110100000085
:10413800F141FF1F0200000012BD00110100000044
:10414800FBBC00110200000062BE0011010000006B
:10415800F041FF1F0200000010BD00110100000027
:104168008861FF1F0200000062BE0011010000000C
:10417800EF41FF1F020000000EBD0011010000000A
:10418800EBBC00110200000062BE0011010000003B
:10419800EE41FF1F020000000CBD001101000000ED
:1041A800E6BC00110200000062BE00110100000020
:1041B800ED41FF1F020000000ABD001101000000D0
:1041C800E1BC00110200000062BE00110100000005
:1041D800EC41FF1F0200000008BD001101000000B3
:1041E800DCBC001102020202020200000000000012
:1041F80016150000A14B0011674B001154BD0011AA
:1042080090011D0018001800FFFF070102030405B4
:104218000602010600000000000000000000000087
:104228000000000000000000000000000000000086
:10423800030000000200000066BE0011010000003B
:1042480074BD00110200000062BE001101000000F0
:10425800AC42FF1F020000007EBD001101000000FB
:10426800B661FF1F0200000060BE001103000000DD
:104278002064FF1F0200000062BE00110100000060
:10428800AC42FF1F020000007CBD001101000000CD
:10429800B861FF1F0200000060BE001103000000AB
:1042A8001864FF1F12A6A6A6000000000000000068
:1042B800161500000001000000000111FFFF0000BA
:1042C8005048593600000000000000000B000500AF
:1042D800F0000000B4000028002800283075A00075
:1042E800A000A000A00000080008E001F0001000F5
:1042F8001000100010001000100050005000500076
:1043080010001000D0070000000000000F0001009E
:104318000500307507001000010081FF0000000053
:10432800FF000000F1730011F9710011896F00118D
:10433800FFFF0100FF0000000D9E0011899B001186
:10434800A19A001100000000000000000000080011
:10435800040000003B0001085902E0018821280000
:10436800FF0000000200000066BE0011010000000E
:104378002CBF00110200000062BE00110100000005
:10438800E943FF1F020000005EBE001101000000AB
:104398000068FF1F0200000062BE0011010000005B
:1043A800E843FF1F020000005CBE0011010000008E
:1043B800E643FF1F0200000062BE0011010000007A
:1043C800E443FF1F020000005ABE00110100000074
:1043D800DC43FF1F180018001D00900102000003B5
:1043E800020200000200000066BE00110100000089
:1043F80040BF00110200000062BE00110100000071
:104408002C44FF1F0200000058BE001100000000ED
:10441800000000000200000060BE00110300000060
:064428002068FF1F20FFC9
:040000051FFF184180
:00000001FF
